:020000040800F2
:2000000000080020652700084522000847220008492200084B2200084D22000800000000E5
:20002000000000000000000000000000512200084F220008000000005322000855220008D0
:2000400057220008592200085B2200085D2200085F22000861220008632200086522000860
:2000600067220008692200086B2200086D2200086F220008712200087322000875220008C0
:2000800077220008792200087B2200087D2200088122000885220008872200088922000812
:2000A0008B2200088D2200088F22000891220008D1220008D3220008D5220008D722000868
:2000C000D9220008DB220008DD220008DF220008E1220008E3220008E5220008E7220008D0
:2000E000E9220008EB220008ED22000810B5DFF89C47002800D12FE0DFF8940700680068F8
:20010000804720680A3010BD80B5DFF880070068C178DFF8802752788A420DD38278002A3D
:200120000AD18288002A07D18172DFF86407006840688047002002BD022002BD10B5DFF870
:200140004C47002800D107E0DFF8440700688068804720680C3010BD206801210182002015
:2001600010BD10B5DFF824472068C1784079DFF8282712689269904721688A7A002A07D031
:20018000002805D10879002802D18878002801D0022010BDDFF8F8060068C0688047206849
:2001A0004179C1722068C1780173002010BD10B5DFF8D8160968002803D10220088200206D
:2001C00010BDDFF8D8460020208008787F22104216D1487A810603D5002141F0020121703C
:2001E0004006207809D540F001002070DFF8A006006800698047204610BD00F0FE00F4E771
:2002000000F07F02012AF6D000F07F000228D6D1487900F00F01DFF88826000652F8210085
:2002200005D500F030001028E0D10020DBE700F44050B0F5805FD9D10020D4E770B5DFF870
:200240004C060068017811F07F0102BF417A01F0DF01417254D0022905D14188002902D100
:200260000179002901D0022070BD417921F08005DFF82C460A0654F825204CBF02F0300252
:2002800002F44052DFF80C361B789D42EBD2002AE9D0807A0028E6D0080654F825000BD574
:2002A00000F03000102826D1284601F021FA3021284601F0D0F91EE000F44050B0F5805FF6
:2002C00019D14BF68F7665B9DFF8D80590F82C10002001F03AFA2068304080F44050206097
:2002E00009E0284601F0F4F954F82500304080F4405044F82500DFF8980500684069804737
:20030000002070BD38B5DFF884050268537923F08000DFF88C151C0651F820404CBF04F038
:20032000300404F44054DFF86C552D78A84207D25588002D04D1002C02D0927A002A01D118
:20034000022032BD1A0651F8202042BF48F6BF731A4082F0100204D44BF68F731A4082F4A9
:20036000805241F82020DFF82805006880698047002032BD80B5DFF814050068417A41F08E
:2003800020014172DFF808050068C0698047002002BDDFF8F8241268538A20B98888C01A61
:2003A000108200207047086818187047F8B5DFF8DC54286800F110042688A168080015D090
:2003C000A6B1A088864288BF06463046884707462088801B2080608830186080002001F0AD
:2003E000A6F932460146384602F0AAF8208860B1DFF8B4044FF4405101800021002001F0BE
:200400009DF9DFF8A8043021018028682188A288914202D303210172F1BD002901D0052181
:20042000F9E706210172DFF88804006880B2DFF88414002241F81020DFF87004302101802E
:20044000F1BD38B5DFF844442068457801787F2211422CD1092D02D1FFF756FE38E0052D56
:200460000BD1C178802906D2817821B9818811B9807A002839D0082045E0032D0AD1C17884
:20048000012926D1818821BB407A800621D5FFF771FF1DE0012D1CD1C178012919D181884C
:2004A000B9B9407A800614D5FFF7C8FE10E001F07F00012804D10B2D0BD1FFF752FE07E046
:2004C000022806D1012DEFD0032D02D1FFF71AFF58B12846DFF8C0130968496988470328DE
:2004E00008BF09200FD00028C5D10620DFF8C013096889B2DFF8BC23002342F81130DFF8C8
:20050000AC1330220A802168087231BD2DE9F041DFF8784320684178062919D101787F2202
:20052000114236D18078012802BFDFF86C030068C16979D0022802BFDFF85C030068016A6A
:2005400072D0032825D1DFF850030068416A6BE0002945D14188E1B9C188022919D1017936
:20056000B9B901787F22114204D1828812B9DFF8481359E001F07F02012A16D10021407929
:20058000C54A12689269904718B92068807A0028EDD120684078C0490968096988470328A1
:2005A0004BD12068092101729BE001F07F010229EFD1407900F00F0100F07002B84B0006FF
:2005C00053F821004CBF00F0300000F44050B14B1B789942DDD2002ADBD10028C7D1D8E792
:2005E000082905D100787F210842D2D1B3491BE00A29CED1017801F07F010129C9D1817A7D
:200600000029C6D041880029C3D101790029C0D1C1880129BDD1002140799F4A1268926928
:2006200090470028B5D1A6490800B2D0206800224282816100208847002021680A8A4FF6FB
:20064000FF739A4202D1092008724AE0022800D00AB90820F8E7087800063CD5C88890422F
:2006600038BF08828C48006890F82C00888201F11005288828B9097A042904BF0726102097
:2006800024D0AF88874205D30426B84288BF3846074600E00226B8B2A96888478046002020
:2006A00001F044F80146BAB2404601F035FFB9B2002001F043F82888C01B28806888381885
:2006C0006880302078494FF440520A80774908802068067205E00320087273484FF4405169
:2006E0000180BDE8F08138B576487149096889B2754A32F8111000EB4100644C21680A7A5F
:20070000092A14D010F8012B0A70216810F8012B4A70851C35F8040B01F060F82168488026
:20072000288801F05BF821688880A888C8802068012101722068C08810B9FFF782FE01E0AF
:20074000FFF7E4FEBDE831406FE02DE9F0414F4C2068017A022901D0042934D100F1100543
:20076000288820B9042904BF0726102024D0AF88874205D30426B84288BF3846074600E0C1
:200780000226B8B2A96888478046002000F0CEFFBAB20146404601F0BFFEB9B2002000F0E2
:2007A000CDFF2888C01B288068883818688030203D494FF440520A803C49088020680672D0
:2007C0002068007A14E0062911D1417805290AD101787F22114206D1C07800F040F82C4838
:2007E0000068006A80472C48006880688047082021680872BDE8F04117E010B5234C206821
:20080000007A032801D0052804D1FFF7CFFD2068007A06E0072803D11F480068C0688047F5
:20082000082021680872BDE8104080B51D4890F82C10002000F089FF14480068017A082932
:2008400006D119494FF480520A80184910220A80007A092801D1012002BD002002BDF0B4C3
:200860000C49097800220E4B59B11C4648F68F7526682E40D7B23E4344F8046B521C8A428E
:20088000F6D340F08000D864F0BC70474C1C0020541C0020100B0020501C0020941C002091
:2008A000005C0040000A00209C1C00209E1C0020505C004004600040AF010008ED00000883
:2008C0003D010008006000400860004070470000F0B5046842688368C0680C604A608B6004
:2008E000C860DFF8BC550A26DFF8B875C0F3074C1CF807C0C0F3072E1EF807E04FEA0E4E59
:200900004EEA0C6C5FFA80FE1EF807E04CEA0E2C4FEA106E1EF807E04EEA0C0C55F804EBA3
:200920008EEA0C0C8CEA040462405340584041F8104F4A608B60C860761ED7D1F0BDC7E7F0
:200940002DE9F04F02F2A002036852F8044B84EA030E436852F8044B84EA0308836852F837
:20096000044B84EA0309C06852F82C3983EA000C09201B23DFF830454FEA1E652D5DCCF3A6
:200980000746365D360446EA0565C9F30726365D45EA06255FFA88F6365D354316697540B7
:2009A0004FEA1866365DCEF307473F5D3F0447EA0666CCF307273F5D46EA07265FFA89F7A3
:2009C0003F5D3E4357697E404FEA19673F5DC8F3074A1AF804A04FEA0A4A4AEA0767CEF375
:2009E000072A1AF804A047EA0A275FFA8CFA1AF804A04AEA0707D2F818A08AEA07074FEA9A
:200A00001C6C1CF804C0C9F3074919F804904FEA094949EA0C6CC8F3072818F804804CEADB
:200A2000082C5FFA8EFE1EF804E04EEA0C0CD2F81CE08EEA0C0C05F07F3E25F07F384FEA46
:200A4000D81803FB08F888EA4E0E0EF07F382EF07F394FEAD91903FB09F989EA480808F069
:200A60007F3928F07F3A4FEADA1A03FB0AFA8AEA490989EA050585EA080A85EA0E0B88EA00
:200A80000E0E89EA0E0E8EEA3B6E8EEA3A4E8EEA352E06F07F3526F07F384FEAD81803FB11
:200AA00008F888EA450505F07F3825F07F394FEAD91903FB09F989EA480808F07F3928F04B
:200AC0007F3A4FEADA1A03FB0AFA8AEA490989EA060686EA080A86EA050B88EA050589EAF8
:200AE000050585EA3B6585EA3A4585EA362807F07F3527F07F36F6095E4386EA450505F05C
:200B00007F3625F07F394FEAD91903FB09F989EA460606F07F3926F07F3A4FEADA1A03FBC1
:200B20000AFA8AEA490989EA070787EA060A87EA050B754089EA050585EA3B6585EA3A4539
:200B400085EA37290CF07F352CF07F36F6095E4386EA450505F07F3625F07F37FF095F43CC
:200B600087EA460606F07F3726F07F3A4FEADA1A03FB0AFA8AEA470787EA0C0C8CEA060A3D
:200B80008CEA050B75407D4085EA3B6585EA3A4585EA3C2C103A401E7FF4EEAE4FEA186021
:200BA000005DCEF307431B5D1B0443EA0060CCF307231B5D40EA03205FFA89F31B5D184353
:200BC000536958404FEA19631B5DC8F307452D5D2D0445EA0363CEF307252D5D43EA052371
:200BE0005FFA8CF52D5D2B4395696B404FEA1C652D5DC9F30746365D360446EA0565C8F30B
:200C00000726365D45EA06255FFA8EF6365D3543D66975404FEA1E66365DCCF307473F5DE5
:200C20003F0447EA0666C9F307273F5D46EA07265FFA88F73C5D3443126962400A604860DA
:200C40008B60CD60BDE8F08F2DE9F047036814686340446855686C40856896687540C068A4
:200C6000D66886EA000802F1100009221B268D4F4FEA136C1CF807C0C4F3074E1EF807E0D7
:200C80004FEA0E4E4EEA0C6CC5F3072E1EF807E04CEA0E2C5FFA88FE1EF807E04EEA0C0C89
:200CA0004FEA146E1EF807E0C5F3074919F807904FEA094949EA0E6EC8F3072919F80790FF
:200CC0004EEA092E5FFA83F919F8079049EA0E0E4FEA156919F80790C8F3074A1AF807A0B5
:200CE0004FEA0A4A4AEA0969C3F3072A1AF807A049EA0A295FFA84FA1AF807A04AEA0909E5
:200D00004FEA186818F80780C3F30743DB5D1B0443EA0863C4F30724E45D43EA0423ECB27F
:200D2000E45D44EA03082CF07F33DB0973430CF07F348CEA44055D4093EA440383EA3563FD
:200D400083EA3C4383EA3C2350F8044B63402EF07F34E40974430EF07F358EEA450C84EA43
:200D60000C0C94EA450484EA3C6484EA3E4484EA3E2450F8045B6C4029F07F35ED097543F8
:200D800009F07F3C89EA4C0E85EA0E0E85EA4C0585EA3E6585EA394585EA392550F804CBA4
:200DA0008CEA050528F07F3C4FEADC1C06FB0CFC08F07F3E88EA4E098CEA09098CEA4E0CD0
:200DC0008CEA396C8CEA384C8CEA382C50F804EB8EEA0C08521E7FF44BAF220ED25DC5F36D
:200DE0000746F65D360446EA0262C8F30726F65D42EA0622DEB2F65D3243466872402E0E02
:200E0000F65DC8F3074C1CF807C04FEA0C4C4CEA0666C3F3072C1CF807C046EA0C265FFAE4
:200E200084FC1CF807C04CEA0606D0F808C08CEA06064FEA186C1CF807C0C3F3074E1EF84A
:200E400007E04FEA0E4E4EEA0C6CC4F3072E1EF807E04CEA0E2C5FFA85FE1EF807E04EEAFC
:200E60000C0CD0F80CE08EEA0C0C1B0EDB5DC4F30744E45D240444EA0363C5F30724E45D92
:200E800043EA04235FFA88F4E45D23430068584008604A608E60C1F80CC0BDE8F0870000E1
:200EA000300A0020000800200009002080B500F0B5FCC049087001BD2DE9F04106460C468D
:200EC000B04614F003000BD04FF6FC702040001D844205D2FF22011BB748201801F0C4FA4C
:200EE000002744B1B44D7959304600F0B5FC361D3F1DA742F7D3B1480021418234B1418AFD
:200F000018F8012B51184182641EF8D1418A028A91420CBF00210321C172BDE8F081A748AC
:200F2000022181720021C172A5480170704710B5A4484168A44C216061600068083801F00D
:200F40003FFA6068BDE810400047000030B587B09E484178491E072900F22581DFE811F0A2
:200F6000260023019100E60001010E01220008001422974901A801F04CFA964800788DF8A4
:200F800008001422A02101A801F0C6FA1421012000F0D4FB3021012000F05DFB8E4803212F
:200FA000017005E185480721017301E1834CA17A022901D005295BD182796AB9C17959B9E5
:200FC000012060620620A072E07A207000206070608006202071E9E07F490B78CBB9C378B2
:200FE000857845EA03232362C37942EA0322A2614279007940EA02202082A069E0610020FE
:20100000E081012008704FF44051022000F035FBCEE0724D206A90B9002100F029FF2878A7
:2010200020732879E978090441EA0060A97840EA01206978084360610320A072CAE7E089DB
:201040000019A269412A0BD340222946283001F0D3F9E0894030E081A0694038A061D2E7C8
:201060002946283001F0C8F90320A07220719DE00A20A0720F2020700020607060800A20BF
:20108000A8E74E4CA07A032818D0042802D0062845D03EE0607BC00741D50520A07220711B
:2010A000002060706080E07A2070607B00F0FE0060730021012000F0DBFE30E0607BC1071C
:2010C0000CD50520A0722071002060706080607B00F0FE006073E07A2070EAE70421A17208
:2010E0002171217B412901D0512901D1502100E0002100919DF8001061709DF80110A1700B
:201100009DF80210E170E17A217040F00200607305E02071002060706080E07A207006228E
:20112000A021204601F0F8F9062130E7234CA07A0A2808D10220A07200202060022020714D
:20114000002060710BE00A20A0720E2020700020607060800A202071002060710E20E072BD
:2011600024E0164CA07A6072E07A20720222A02104F1080001F0D0F9022108E70F4CA07A0E
:20118000801E012804D9C01E012801D9001F0DD10220A07200202060022020710020607155
:2011A0002062A061DBE7022000F01CFE00F009FE07B030BDA61C00203C130020140B002093
:2011C000651C002000400008881C0020681C0020E0F7FF1F203C0008641C0020F01B00209A
:2011E00010B49348016842688068D9B1914B9970C1F307241C71C1F307449C71090E1972CC
:201200009A72C2F307211973C2F307419973110E19749874C0F307211975C0F30741997526
:20122000000E187610BC704780B583480068807A40B1012000F05CFA022000F049FA7F48B9
:201240000021017001BD000038B5FFF7C9FF7A4C20680021817201F0CFF9794800214160F5
:201260004FF40441774A1180016020687649C9794172764D2068807A60B92878012804D1FB
:201280004FF4FA71042000F0F3FD00BF2068807A0028F2D06E480521017031BD10B56D48BC
:2012A00000218172002000F0C7F94FF40071002000F0C9F92021002000F0CDF9202100204C
:2012C00000F02DFA644C94F82C10002000F03DFA6021002000F022FA002000F0EDF9002075
:2012E00000F0E0F90021012000F0ADF9A021012000F014FA2021012000F0ADF90021012033
:2013000000F0BBF90021022000F09DF9E021022000F005FA94F82C10022000F016FA4FF421
:201320004051022000F0A9F90021022000F093F90021032000F087F94FF48071032000F0AE
:20134000EDF92021032000F086F90021032000F094F994F82C10002000F0F7F9002000F03B
:20136000A1F90020FFF77BFA34480021017010BD7047704780B5304909680A7802F07F02EB
:20138000212A0DD1FE280BD14888002808D18888002805D1C888012802D13048020001D1AB
:2013A000022002BD88610020488200F037F8002002BD80B5204909680A7802F07F02212A2C
:2013C00018D1FF2816D14888002813D18888002810D1C88800280DD1012000F089F9022016
:2013E00000F076F9032000F083F9144800210170002002BD022002BD01B900B1022070470D
:201400001749FEF7C6BF1749FEF7C3BF0A490968C978154A02EBC101FEF7BBBF002805D19B
:201420000548006801210182002070470F487047E8F7FF1FA40A00204C1C0020641C00207A
:20144000405C0040A41C002050260008A01C0020A81C0020301C0020000A00201D140008C3
:20146000F80A0020000B0020580A0020981C00202DE9F84F4BF68F78684D48F60F7B40F671
:201480008F77674CDFF89C91DFF89CA123E0300404D5206838402060FFF7AFF9206808EAD3
:2014A00000002988CA0448BF80F48050890444BF80F4005080B22060206848F6BF7108401E
:2014C0006988CA0648BF80F01000890644BF80F0200080B22060606CAAF80000000460D549
:2014E00047F6FF706064BAF8000010F00F0089F8000035D1206800F440502880206800F008
:2015000030006880206808EA000080F400502060206848F6BF71084080F020002060BAF8F5
:201520000000C00620680FD40BEA00002060FFF70CF920684FF408410842AFD0206838402D
:201540002060FFF7D0F8A9E786B2300605D520680BEA00002060FFF7F8F8300597D5EDE71D
:2015600054F820108EB231040AD554F82010394044F820102D4901EB800050F8040C804739
:201580003006A8D599F8000054F820100BEA010144F82010264901EB800050F8040C80472E
:2015A00099E7BDE8F18F2DE9F84FDFF8809040F68F75DFF86CB01B4F47F6FF781A4CDFF8BA
:2015C00074A024E0CAF80080208800F00F0038705BF820108EB2310409D55BF820102940A0
:2015E0004BF8201009EB800050F8040C804730060DD538785BF8201048F60F7211404BF847
:2016000020100B4901EB800050F8040C8047DAF8000020800004D5D4BDE8F18F9C1C00209F
:20162000005C0040A71C0020A21C0020DC0A0020C00A0020445C00404FF6F8710840DFF8B0
:2016400084110860704710B4DFF87C2152F8203048F68F145CE010B4DFF86C2152F8203025
:2016600048F6BF742340CC0648BF83F01003890644BF83F020039BB210E010B4DFF84821CE
:2016800052F820304BF68F742340CC0448BF83F48053890444BF83F400539BB242F82030B7
:2016A00010BC7047DFF8201151F820204BF68F731A4082F4405208E0DFF80C1151F820200C
:2016C00048F68F6300E000001A4041F820207047DFF8F41051F82020520408D551F8202050
:2016E00048F68F731A4042F4804241F820207047DFF8D41051F82020520608D551F8202026
:2017000048F68F731A4042F0400241F8202070472340194342F8201010BC704738E0294A54
:20172000126892B202EBC000284A37E03BE02549096889B201EBC00024493AE0214A126868
:2017400092B202EBC000224A2AE01E4A126892B202EBC0001F4A02EB40003F2909D34A0922
:201760001F23194204BF521E92B2910241F4004105E04A08C90744BF521C92B2910201609C
:2017800070471049096889B201EBC000114914E00C4A126892B202EBC0000F4A49084900DF
:2017A00042F8101070470749096889B201EBC000094951F8100080B2704751F810008005FE
:2017C000800D7047505C0040005C004008600040046000400C600040006000400106090C89
:2017E00041EA102070470000DFF854110A6802F03802FFE70A600A68104308607047DFF8F2
:2018000040110A6822F01002F4E7DFF83801DFF838110160DFF834110160704770B50546D1
:2018200040F6FF76304600F09BF8042813D1484C206840F0020020606560206840F0400069
:201840002060304600F08CF8012804D0216841F6FD721140216070BD70B505460E4616F128
:20186000010F01D1042070BD0F2000F079F8042816D1374C206840F0010020602E800F20F9
:2018800000F06EF8042804D1300C68800F2000F067F8012804D0216841F6FE721140216050
:2018A00070BD70B5044640F6FF75284600F058F8042830D1274E2448306024483060B06882
:2018C00040F02000B060B06840F04000B060284600F046F8042817D1B06841F6DF71084079
:2018E000B060B06840F01000B0601B48002C14BF0021A5210180284600F032F801280AD01B
:20190000B16841F6EF7204E0012804D0B16841F6DF721140B16070BD10480168C90701D59E
:20192000012070470168490701D5022070470068C00601D5032070470420704700000000AE
:20194000002002400420024023016745AB89EFCD102002400820024000F8FF1F0C2002409F
:2019600038B50546FFF7D8FFFF2408E00098401E009000980028F9D1FFF7CEFF6D1E0128D0
:2019800004D125B1002000900094F2E705B9052032BD000058480021C16001611421416192
:2019A00000218161C161016841F0010101604168524A114041600168514A114001600168AF
:2019C00021F480210160416821F4FE01416000218160704748490A6822F480320A600A6832
:2019E00022F480220A60B0F5803F03D0B0F5802F04D07047086840F4803002E0086840F4D5
:201A0000A0200860704710B53E4C312000F05DF820706068401C6060207810B96068FF283E
:201A2000F3D1312000F051F8401E8041C043C00F10BD354A136823F47C13184308431060E4
:201A400070473249086070472F490A68920850EA8200086070472C48006800F00C00704747
:201A600029490A6822F0F00203E027490A6822F4E06210430860704723490A6822F4605249
:201A800042EAC00008607047214908607047214A0029116814BF084321EA00001060704755
:201AA0001D4A0029116814BF084321EA0000106070471A4A0029116814BF084321EA00009E
:201AC0001060704716490870704741090A4A012908BF116803D002290CBF116A516A012227
:201AE00000F01F0002FA00F00840401EFFE78041C043C00F70470000001002400000FFF8CC
:201B0000FFFFF6FE801C00200410024060004242D8004242181002401C1002400C1002404B
:201B20000710024080B50620FFF7CCFF4FF48070ADF8000018208DF8030003208DF80200EE
:201B400000A94948A6E080B5FFF724FF4FF48030FFF740FFFFF757FF012828D11020FFF7BB
:201B60004EFE0220FFF740FE0020FFF779FF4FF48060FFF781FF4FF48060FFF776FF0020EE
:201B8000FFF782FF4FF4E0114FF48030FFF751FF0120FFF756FF3920FFF797FF0028FAD01E
:201BA0000220FFF751FFFFF756FF0828FBD1FFF72CFE01212020FFF76AFF01214FF4000030
:201BC000FFF76EFF01214FF40170FFF760FFBDE80140A7E780B500F04DF8BDE8014000F0C3
:201BE00019B980B500214FF0006000F0C1FA1F48002101604FF4A06000F076FA14208DF82E
:201C0000000001208DF8010000208DF8020001208DF8030000A800F06CFA13208DF8000017
:201C200000208DF801008DF8020001208DF8030000A800F05EFA1B208DF8000000208DF879
:201C400001008DF8020001208DF8030000A800F050FA01BD064A00284FF48071104601D0E0
:201C600000F0DEB900F0DAB900080140445C00400014014080B54FF48070ADF8000014209B
:201C80008DF8030003208DF8020000A9004801E00014014000F062F901BD000000B583B0FA
:201CA0004C4801788DF8001040788DF801004A48017A8DF80210417A8DF80310817A8DF8CD
:201CC0000410C07A8DF80500062100A800F067F803B000BD10B582B0404C607800F2001041
:201CE000ADF800000222A02100A800F015FC0320207002210120FFF721FD30210120FFF73E
:201D0000AAFC13BD80B535480178022906D0032901D0042907D1BDE8014052E00079F32873
:201D200008BFFFF713F901BD10B50220FFF729FD04462246E0212A4800F002FC274801781E
:201D400011B1012904D007E02046BDE8104007E00079F32803D11EE0022000F043F810BD1A
:201D600010B51E4C20B102461D49201D00F044FB2079F12804D0F32805D0F52804D006E0FC
:201D8000BDE810408AE706E0BDE81040A2E70220BDE8104026E0BDE81040FFF7D7B810B51D
:201DA0000C462246A02100F0B7FB21460120FFF7C5FC30210120FFF74EFC08480321017030
:201DC00010BD0648002101704FF440510220FFF754BC0000FE3F00081C270008641C00202A
:201DE000F01B002080B518B1022807D00AD301BD10210120BDE80440FFF72DBC10210120B2
:201E0000FFF729FC4FF480510220BDE80440FFF734BC000000B585B001214FF40060FFF7FD
:201E200036FE01210420FFF732FE00F0FBF8464802210186018801F09F0101800188018042
:201E40006020ADF800000220ADF808000120ADF8020000A800F0F3F8012000F02AF90120EE
:201E600000F024F9012000F00EF905B000BD000070B582B004460D46344E3078844207D010
:201E80000021042000F003F9002000F0F8F802E07068A84257D0062C3DD8DFE804F0040E32
:201EA000122314212B002A48016821F0F0010091009941F0400101602DE0502000F0F1F85D
:201EC00029E04020FAE7502000F0EBF82148858248F6A04101820121042000F0D8F81AE063
:201EE0004020F1E71B4864218182818A49080184642106E017488582C5F34F0101844FF63B
:201F0000FF7101820188C9B20091009941F4D041009100990180104801210160307818B163
:201F2000042801D0052809D144B10948016821F0F0010091009941F0B00101603470756006
:201F4000012000F09CF873BD002C0140781C002004080140182C0140808225422DE9F04109
:201F6000CB7803F00F02DB0644BF8B781A430B88DCB22CB3D0F800C0002401250F2605FAD0
:201F800004F707EA0308B84515D14FEA840E06FA0EF82CEA080C02FA0EFE4EEA0C0C91F88B
:201FA00003E0BEF1280F08BF476191F803E0BEF1480F08BF0761641C082CE0D3C0F800C069
:201FC0004FF48074A34227D3D0F804C0002401250F2604F1080705FA07F707EA0308B845E6
:201FE00015D14FEA840E06FA0EF82CEA080C02FA0EFE4EEA0C0C91F803E0BEF1280F08BF8F
:020000040800F2
:20200000476191F803E0BEF1480F08BF0761641C082CDED3C0F804C0BDE8F0810161704767
:202020004161704780B501214FF40060FFF741FD00214FF40060BDE80440FFF73ABD10B4BB
:20204000DFF884100A88DFF8843000241C60D2B2048842EA04220A8042881A6082889A6024
:2020600002895A604289DA60DFF86420FFE783891360C3895360C088088410BC7047DFF829
:20208000541008607047DFF8501008607047DFF84C20012911880CBF084321EA00001080B0
:2020A000704709490A8840F67F7308E00C49086070470C49086070470A884FF2FF331A402E
:2020C00042EA002008807047182C014010842542A880254200802542BC8825420C2C01405B
:2020E0001C8025422C832542264908432649086070472DE9F04105780121C2787AB3224AC6
:20210000126802F4E062C2F5E062120AAB10DFF8708058F8237005F00305ED00FF26AE4096
:20212000B7434478C2F1040E04FA0EFC90F802E00F2424FA02F202EA0E0242EA0C02120124
:20214000AA4032403A4348F82320007842110F4B00F01F0001FA00F043F8220006E0681148
:20216000064A05F01F03994042F82010BDE8F081074A1140084307490860704780E100E002
:2021800000E400E00000FA050CED00E000E100E080FFFF1F08ED00E070B5FFF7D4FCFFF78F
:2021A00019FDFFF71EFD4FF4FA610420FFF760FE0120FFF776FB00F0D3F900210120FFF766
:2021C00057FEFEF7ACFE1848184C194D194E01780529FCD12878800720D52078212809D030
:2021E000412802D0512808D012E013480068FEF75DFE0DE0512020700AE0326892B20F4940
:202200000F4800F075F831680B480068FEF754FE287800F0FD0040F0010028702078072852
:20222000D8D1FEF784FED5E7A81C0020200B0020210B0020300B0020280B00203C1300202A
:202240003C0B00207047FEE7FEE7FEE7FEE77047704770477047704770477047704770475D
:2022600070477047704770477047704770477047704770477047704770477047FFF793B91A
:2022800000F026B970477047704770477047704781B00C48018821F0040101800A480168C5
:2022A000491C01600948026822F0F0020092C90700994CBF41F0400141F0B001016001B02D
:2022C00070470000102C0140901C00200408014070477047704770477047704770477047F9
:2022E00070477047704770477047704770470000F0B585B005460E4617460F20074200D1BE
:202300000FB901202FE0194C2078F8B900A9184A135C01F8013B401C0428F9DB042001A93E
:20232000144A135C01F8013B401C1028F9DB211D1148FEF7CDFA221D00A900A8FEF784FCDB
:20234000211D00A8FEF7FBFA0120207057B1221D31462846FEF7F4FA10351036103FBFB2A2
:20236000002FF4D1002005B0F0BD00003C1B0020E0F7FF1FE4F7FF1F4427000830BF704769
:2023800020BF704740BF7047BFF36F8F7047BFF34F8F7047BFF35F8F704701DF7047EFF373
:2023A0001480704780F31488BFF36F8F7047EFF30980704780F309887047EFF3088070475E
:2023C00080F30888704762B6704772B67047EFF31080704761B6704771B67047EFF313804B
:2023E000704780F311887047EFF31280704740BA704700BA704700004AB38B0707D011F8A7
:20240000013B00F8013B521E21D08B07F7D183071ED1103A07D330B4B1E83810103AA0E85D
:202420003810F9D230BC530724BFB1E80810A0E8081044BF51F8043B40F8043BD20724BF51
:2024400031F8022B20F8022B44BF0B7803707047083A07D3B1E80810083A40F8043B40F873
:2024600004CBF7D25307E4E762F30F2262F31F42401810F0030308D0C91A1FD3DB0748BF6F
:2024800000F8012D28BF20F8022D130030B414461546103928BF20E93C00FAD8490728BFBE
:2024A00020E90C0048BF40F8042D890028BF20F8022D48BF00F8012D30BC7047C91818BF58
:2024C00000F8012DCB0728BF00F8012D7047000038B50D4C0D48016861800D4D61882A8866
:2024E0001140490505D54FF6FF310160094840688047608829880840000403D5FEF7B8FF64
:202500000120207031BD00BFA01C0020445C0040A41C0020000A002010B4104B03EB410148
:20252000521C52100AD010F8013B10F8014B43EA042321F8023B891C521EF4D110BC704752
:20254000064B03EB4101521C521005D051F8043B20F8023B521EF9D17047000000600040E7
:2025600010B50A4CE461022020720948206209496162006880474FF40070E0624FF4801068
:20258000A0624FF40060206310BD00BF301C0020000A0020800A002080B500F0EFF8020039
:2025A0000023DB431068984204D011000220ABBE002010605068984204D0111D0220ABBE69
:2025C0000020506001BD000010B40FE001680918001D50F8042BD40744BFA9F10104A21865
:2025E00051F8044B42F8044B1B1FF9D150F8043B002BEBD110BC704780B50120FFF72AFB54
:202600000648012101600021016041604FF40441034A11800160002002BD0000405C004044
:20262000A41C002010B5084979441C31074C7C441A34A14206D0081D0A685118884701466A
:20264000A142F8D110BD00BF7C0000009C0000000902270001010080320904000003FFFF36
:20266000FF04070581024000000705020240000007058302400000002603530054004D004A
:202680006900630072006F0065006C0065006300740072006F006E006900630073000000F2
:2026A0000BE050F8041BCB0744BFA9F101035918002341F8043B121FFAD150F8042B002AAC
:2026C000EFD17047DDFFFFFF98110000140B002000000000F5FEFFFF14030000C0000000F9
:2026E00000080020000000001A03530054004D00330032002000530054004C0069006E0052
:202700006B00000000F048F8002801D0FFF78AFF0020FFF741FD00F039F80000120100021C
:202720000000004083044837000101020301000080B5FFF731FF024A11001820ABBEFBE710
:20274000260002004920616D206B65792C2077617761776110035300540020004C0069004E
:202760006E006B00C046C046C046C046FFF7CAFF07463846FFF7DCFFFBE70000004870472C
:20278000080B0020FFF7BEBAFFF7CEBA80B5FFF7EFBF00000403090401207047637C777B84
:2027A000F26B6FC53001672BFED7AB76CA82C97DFA5947F0ADD4A2AF9CA472C0B7FD932602
:2027C000363FF7CC34A5E5F171D8311504C723C31896059A071280E2EB27B27509832C1AFF
:2027E0001B6E5AA0523BD6B329E32F8453D100ED20FCB15B6ACBBE394A4C58CFD0EFAAFBFB
:20280000434D338545F9027F503C9FA851A3408F929D38F5BCB6DA2110FFF3D2CD0C13ECA6
:202820005F974417C4A77E3D645D197360814FDC222A908846EEB814DE5E0BDBE0323A0AEC
:202840004906245CC2D3AC629195E479E7C8376D8DD54EA96C56F4EA657AAE08BA78252E1D
:202860001CA6B4C6E8DD741F4BBD8B8A703EB5664803F60E613557B986C11D9EE1F8981165
:2028800069D98E949B1E87E9CE5528DF8CA1890DBFE6426841992D0FB054BB1652096AD5EA
:2028A0003036A538BF40A39E81F3D7FB7CE339829B2FFF87348E4344C4DEE9CB547B9432B1
:2028C000A6C2233DEE4C950B42FAC34E082EA16628D924B2765BA2496D8BD12572F8F66487
:2028E00086689816D4A45CCC5D65B6926C704850FDEDB9DA5E154657A78D9D8490D8AB0029
:202900008CBCD30AF7E45805B8B34506D02C1E8FCA3F0F02C1AFBD0301138A6B3A9111418B
:202920004F67DCEA97F2CFCEF0B4E67396AC7422E7AD3585E2F937E81C75DF6E47F11A7137
:202940001D29C5896FB7620EAA18BE1BFC563E4BC6D279209ADBC0FE78CD5AF41FDDA83309
:202960008807C731B11210592780EC5F60517FA919B54A0D2DE57A9F93C99CEFA0E03B4D9A
:20298000AE2AF5B0C8EBBB3C83539961172B047EBA77D626E169146355210C7D491200082C
:2029A0009D120008711300087313000875130008B3130008F9130008011400080714000894
:2029C0000D140008000000004000000000000001000000020000000400000008000000106F
:2029E0000000002000000040000000800000001B0000003694270008040000007826000839
:202A000026000000E82600081A000000A40A00201A0000005427000810000000CD08000808
:202A200029120008CD080008CD080008CD080008CD080008CD080008CD080008CD08000848
:202A40001A0330003000300030003000300030003000300030003000310000008527000864
:202A6000CD080008CD080008CD080008CD080008CD080008CD080008CD0800088927000893
:202A8000CD080008CD080008CD080008CD080008CD0800081C27000812000000502600080A
:202AA00027000000FFFFFFFFFFFFFFFF0401000000010020412B0008652B0008652B00082D
:202AC000652B0008652B0008652B000800000000000000000000000000000000652B000896
:202AE000652B000800000000652B0008652B000810B5084979441C31074C7C441A34A142AA
:202B000006D0081D0A68511888470146A142F8D110BD00BF080000000400000000F020F87D
:202B2000002801D0FFF7E4FF002000F017F800F012F8000001491820ABBEFBE726000200B5
:202B4000C046C046C046C046FFF7E8FF07463846FFF7F0FFFBE780B5FFF7F8BF0020704735
:202B600001207047FEE7FFFFFFFFFFFFFFFFFFFFFFFFFFFFFFFFFFFFFFFFFFFFFFFFFFFFB2
:202B8000FFFFFFFFFFFFFFFFFFFFFFFFFFFFFFFFFFFFFFFFFFFFFFFFFFFFFFFFFFFFFFFF55
:202BA000FFFFFFFFFFFFFFFFFFFFFFFFFFFFFFFFFFFFFFFFFFFFFFFFFFFFFFFFFFFFFFFF35
:202BC000FFFFFFFFFFFFFFFFFFFFFFFFFFFFFFFFFFFFFFFFFFFFFFFFFFFFFFFFFFFFFFFF15
:202BE000FFFFFFFFFFFFFFFFFFFFFFFFFFFFFFFFFFFFFFFFFFFFFFFFFFFFFFFFFFFFFFFFF5
:203C000026F1DDF3D15E7CAF665B84BE7BB5E9249F00000034EF180068EE180000000000DB
:203C20004DEE1800F95AA676481C01B2F408FC0100000000000000000000000000000000B2
:203C4000940AFC01D80AFC0108000000800BFC0100000000280CFC0100000000980CFC0188
:203C60000000000000000000D007FC01C0EE18005869A676D007FC010000000030F01800C1
:203C80000B8CA5760100000000000000E983A576481C01B23400000000200000F00BFC0187
:203CA00000000000010000000000000000000000B00CFD0100000000000000001C0000002D
:203CC000980AFC01900AFC0100000000D80AFC01EB05A676D007FC010000000000000000EF
:203CE00008000000000000004CEF18008C2BA67600000000D007FC010000000000000000C2
:203D000050EF1800AD6AA67601000000481C01B26CEF18004674A576D007FC0100000000E5
:203D200001000000481C01B2100BFC01B4EF18002842A676481C01B2F408FC01EC08FC0111
:203D4000F408FC0100000000D007FC0101000000E80AFC01100BFC01ACEF18005869A676FE
:203D600000000000D007FC01CCEF18000B8CA5760100000000000000537AA576481C01B2EA
:203D800000200000000000000100000018F0180065541375481C01B21008FC01080000006D
:203DA00000000000FFFFFFFFD007FC010000000014F0180040F018000000000000000000CF
:203DC000000000006CF01800501959007E15005FCCEF18000900800164F01800E24C13753C
:203DE000481C01B2C06DA200080000004CF01800506AA6761CC0AA7601000000EF7AA5762A
:203E0000481C01B2340000000020000064F01800104D13756CF01800481C01B2481C01B244
:203E200000000000704F347601000000D0F018005CFD0575040000001C000000000000004D
:203E4000D0F0180073FD057500030A7500000000655A0475481C01B2B8F01800560C047534
:203E600003000000BCF0180000000000000000000000000000000000FFFFFFFF020000007D
:203E800024F118000000000001000000481C01B284F1180063680775481C01B2850010015C
:203EA000705E0775C06DA200080000001C0000000400000034000000100000000202000079
:203EC00000000000A8BF5900000200002D52347601000000A8BF5900000000000F0001B274
:203EE0002100F00003000000030000006900000014000000730010010300000003000000A4
:203F00006600000011000000730010010000000088F11800340000000D000000806CA20046
:203F200000000000030000000800000085001001C06DA20034000000020200000E000000CB
:203F400000000001C8F118002A6D07750000000015020000A5AB0575030000000000000098
:203F6000A8BF5900806CA2000100000001000000C8F1180000000000EB0300004CFF4700A0
:203F8000F01C590068FF47004CFF47000CF218005228410011BD0000FCF11800F978400027
:203FA0000000000011BD000000000000FF7840000000000000000000B8070D0024F2180082
:203FC000FDFA40000000000000000000000000000000000085FC180085FC18000000000078
:203FE0006A17005FB8F21800C4DA400011010000EB030000B8070D00000000002C1E240403
:020000040800F2
:204000000008002029C1000819B300081BB300081DB300081FB3000821B30008000000004E
:2040200000000000000000000000000025B3000823B300080000000027B3000829B30008FC
:204040002DB300082FB3000831B3000833B3000835B3000837B3000839B300083DB30008E6
:204060003FB3000841B3000843B3000845B3000849B300084FB3000857B3000861B3000810
:2040800071B3000879B300087DB300087FB3000883B3000887B3000889B300088BB3000844
:2040A0008DB300088FB30008BFB30008C1B3000815B4000817B4000819B400081DB4000826
:2040C0001FB4000821B4000823B4000825B4000827B4000829B400082BB400082DB40008D0
:2040E0002FB4000831B4000833B400080121002801D1802070474FF6F8720240082A06D08D
:20410000302A06D0382A06D0402A06D007E0092133E00B2131E006212FE00A212DE000F038
:204120000700102A01D0182A0DD1012804D0022804D0042804D005E0142104E0152102E03C
:20414000172100E01621202A01D0282A15D1401E062811D8DFE800F0040610080A0C0E004B
:2041600010210AE0112108E0132106E0182104E0192102E01A2100E012210846704710B59F
:20418000040001D0022C07D100220121DFF8F80C07F005F806F003FA022C07D14FF6FF7084
:2041A0000146411889B20029FBD101E0012C01D106F0FBF9802010BD80B506F085FCDFF875
:2041C000340B90F82000012801D100200CE003F088FE802804D103487844083003F001FFC9
:2041E00002BD00BF647F000004F032FBBDE802407CE7000080B506F067FCDFF8F80A90F804
:204200002000012801D10220EEE703F06AFE802804D103487844083003F0E3FE02BD00BF23
:20422000207F000080B503F05AFE802806D1084878441C3000F2101003F0D3FE802806D133
:20424000034878440A3000F2081003F0CAFE02BD306A0000F8B506460C46FFF7CBFFDFF81D
:20426000945A95F82010012909D180284DD100A9304604F01DFBFFF739FF009944E0234F41
:204280007F448837F1B2C95D6970C6F30721C95DA970C6F30741C95DE970310EC95D29715B
:2042A000802808BF03F01DFE802804BF284603F098FE802804BF07F2001003F092FE802880
:2042C00008BF03F00CFE802804BF07F2201003F088FEDFF8006D802804BF304603F003FEF4
:2042E0003178C95D6962696A7278D25D41EA02216962696AB278D25D41EA02416962696AE7
:20430000F278D25D41EA026169629FE1746900002DE9F04105460E46FFF76CFF0446DFF8E6
:20432000D47997F82000012809D1802C68D12946304604F0F0FAFFF7D9FE044660E0DFF8A8
:20434000C880F84408F1C208E8B210F808007872C5F3072010F80800B872C5F3074010F862
:204360000800F872280E10F808003873F0B210F808007870C6F3072010F80800B870C6F36F
:20438000074010F80800F870300E10F808003871802C02D103F0A5FD0446802C03D138460B
:2043A00003F01FFE0446802C04D107F1080003F018FE0446802C04D108F2641003F011FEDE
:2043C0000446802C02D103F08AFD0446802C04D108F2181003F005FE0446802C04D108F2F2
:2043E000201003F0FEFD0446802C04D108F2101003F0F7FD0446052107F1090007F0ACFEC1
:204400002046BDE8F08100BF786800002DE9F04182B004460D46FFF7EDFEDFF8D86896F8E5
:204420002010012912D1802840F08880002070622146284604F0ECFA28B900A9284604F0D2
:20444000AAFA00997162FFF751FE77E0DFF8888B424F7F4407F58377E1B2C95D88F8011032
:20446000C4F30721C95D88F80210C4F30741C95D88F80310210EC95D88F80410802808BF95
:2044800003F02FFD802804BF07F2501003F0A9FD802808BF03F023FD802804BF07F5AB709C
:2044A00003F09FFD802808BF03F01BFD802804BF404603F096FD802806D1E85D88F809002F
:2044C00008F1080003F08DFD802805D1E85D707606F1180003F085FD802804BF07F25C1061
:2044E00003F07FFD802808BF03F0F9FC802804BF07F2201003F075FDDFF8D88A802804D147
:20450000414607F2081003F079FD98F80010C95D7162716A98F80120D25D41EA0221716225
:20452000716A98F80220D25D41EA02417162716A98F80320D25D41EA0261716280280BD1DC
:204540000F2D716A05D1490849006208B1EB420F00E0A14218BF0D20BDE8F681246700000F
:20456000F8B506460C46FFF745FEDFF8885795F82010012909D1802868D100A9304604F04C
:204580000AFAFFF7B3FD00995FE0802808BF03F0A8FC802806D11E487844743000F23C1010
:2045A00003F01FFD802808BF03F099FC802806D1174878445A3000F5A17003F012FD802821
:2045C00008BF03F08EFC802808D1114878444030305C687605F1180003F003FD802806D1A7
:2045E0000B4878442A3000F2481003F0FAFC802808BF03F074FC064E7E441436802804BF82
:2046000006F2201003F0EDFCDFF8C87902E000BF70660000802804D1394606F2081003F008
:20462000EDFC3978895D6962696A7A78925D41EA02216962696ABA78925D41EA0241696235
:20464000696AFA78925D41EA02616962696A2160F2BD00002DE9F04105460C468020DFF86F
:20466000946696F82010012905D1DFF8701909682960002145E0DFF85C790121384603F0A3
:204680003CFBDFF88480F84408F17E08797811F808107162716ABA7812F8082041EA0221DB
:2046A0007162716AFA7812F8082041EA02417162716A3A7912F8082041EA02617162716A6B
:2046C000296080281ED10021384603F016FB797811F808107162716ABA7812F8082041EAC8
:2046E00002217162716AFA7812F8082041EA02417162716A3A7912F8082041EA02617162E3
:20470000716A2160BDE8F081786500002DE9F84F0546DFF8C0484FF00008FFF76BFD012DF0
:2047200007BF21254FF040091525C146DFF8C46596F8201001291ED1802840F099800027B5
:20474000012D14DBDFF8984804E0B8F1000F0AD1202F03D0214607EB090001E02146212001
:2047600004F019F980467F1C241DAF42EDDB4046FFF7BCFC7CE0802808BF03F0B2FB802891
:2047800007D13C48784400F1EC0000F2281003F028FC802808BF03F0A2FB802806D13548E8
:2047A0007844D03000F5977003F01BFC802808BF03F097FB0027012D4DDBDFF8B880F8447B
:2047C00008F1B208C144DFF818A808F2341B802809D1202F0CBF842099F80000707606F193
:2047E000180003F0FEFB802804BF584603F0F9FB802808BF03F073FB802804BF08F2201060
:2048000003F0EFFB802804BF204603F070FB14F8011B11F80810CAF8001014F8012B12F82F
:20482000082041EA0221CAF8001014F8012B12F8082041EA0241CAF8001014F8012B12F844
:20484000082041EA02614AF8041B641C7F1C09F10109AF42BBDB802808BF03F040FB802856
:2048600006D1044878440C3000F2081003F0B9FBBDE8F28F0C64000038B5044600202070EF
:20488000FFF7B8FC80280ED1DFF8685405F12401DFF85007FFF7DEFC802804D1696A89035F
:2048A00044BF0121217032BD2DE9F8438046084616469946089D099C104F7F443E3757F883
:2048C0002810FFF725FD802805D107EB880001692846FFF71DFD80280DD107EB8900006C3B
:2048E00007EB8801096A802C03D107EB8602126B1043FFF70DFDBDE8F28300BFA47400000F
:2049000038B50C46DFF8E016084012B9DFF8DC1605E0012A0CBFDFF8D816DFF8D81641EA1F
:204920000005FFF767FC802807D1084878441C3050F824102846FFF7EBFC802804D1DFF826
:20494000B8160320FFF7E4FC32BD00BFDC760000F8B5044600202070FFF74CFC802808BF3C
:2049600000F07BF8802804D1DFF890160120FFF7CFFC802805D1DFF88816DFF88806FFF7AA
:20498000C7FC0027DFF85C66DA4D802804D105F124013046FFF75EFC696A01F00071491E73
:2049A0008941C943C90F7F1C802808BF002903D14FF47A729742E8DB802802D1002900D102
:2049C000F2BD002705F124013046FFF743FC7F1C696A890105D5802803D14FF47A718F42EE
:2049E000F0DB696A89030BD5802804D13146DFF81806FFF78DFC8028E2D101212170F2BD88
:204A00000021FBE770B5044600202070FFF7F2FB802805D1DFF8CC15DFF8F005FFF778FC25
:204A200080280CD1B34DDFF8BC6505F124013046FFF710FC696ADFF8D825114205D170BD69
:204A400005F124013046FFF705FC802802D1696AC901F5D40121217070BD70B50024FFF7CE
:204A6000C9FB8028A34E18D1DFF878552946DFF89805FFF74DFC802804D106F12401284623
:204A8000FFF7E8FB641C716A890302D5716A090303D5C82C01DA8028E6D0802805D1DFF83E
:204AA0007415DFF84005FFF7D5FB70BD2DE9F84F04460D4690461E460027FFF79BFB06B1C0
:204AC0003460DFF8309299F82010012941D1802840F0B48004F00C00C0F11000800800F067
:204AE0000309C84538BFC146BA46B9F1000F15D0A3464FEA9B0080002FB905EB8A0103F06E
:204B0000D7FE074604E01EB13168A14208BF30600AF1010A0BF1040BCA45EAD304EB890098
:204B200080084FEA800AC1450FD277B9A8EB090205EB8901504603F097FF070005D026B129
:204B40003068A04208BFC6F800A03846FFF7CEFA74E03B4E7E44E836E1B2895D89F80110B2
:204B6000C4F30721895D89F80210C4F30741895D89F80310210E895D89F80410802808BF4B
:204B800003F0AFF9802804BF484603F02AFA802804BF06F2001003F024FA802832D106F243
:204BA000001003F01EFA2DE0A1F10108802829D109F1100106F2001003F020FA99F81010BF
:204BC000895DC9F82410D9F8241099F81120925D41EA0221C9F82410D9F8241099F8122039
:204BE000925D41EA0241C9F82410D9F8241099F81320925D41EA0261C9F82410D9F8241023
:204C000045F8041B1FFA88F10029CDD1802808BF03F065F9802804BF06F2181003F0E1F9C7
:204C2000802804BF06F2201003F0DBF9802805D109F1100106F2101003F0E0F9BDE8F28F87
:204C4000406000002DE9F04182B006460C4606F00305FFF7B1FA274F97F8201001290BD1C3
:204C6000802805D100A9304603F022FEFFF73EFA0099EA00D14037E0DFF87480F84408F1AB
:204C80007008F1B211F808107970C6F3072111F80810B970C6F3074111F80810F970310EFA
:204CA00011F808103971802808BF03F01AF9802804BF384603F095F9802804BF08F20010D5
:204CC00003F08FF9802804BF08F2001003F089F9802805D107F1100108F2001003F08EF964
:204CE000E919097C11F808102170BDE8F68100BF905F0000181B00202DE9F04707460C4672
:204D000015460026FFF776FADFF8588D98F82010012933D180282FD107F00C00C0F1100096
:204D2000800800F00308454538BFA846B146B8F1000F10D0BA4600E03EB954F829104FEA5D
:204D40009A00800003F0E7FD064609F101090AF1040AC145F0D307EB880080088000A845D1
:204D600007D236B9A5EB080204EB880103F0EBFE06463046FFF7BAF9BDE8F087414E7E44A5
:204D800006F58176F9B2895D88F80110C7F30721895D88F80210C7F30741895D88F803102A
:204DA000390E895D88F804102178895D88F809102168C1F30721895D88F80A102168C1F3F8
:204DC0000741895D88F80B102168090E895D88F80C10802808BF03F084F8802823D14046E8
:204DE00003F0FFF81FE06D1E802804BF08F1080003F0F7F8802816D154F8041FC9B2895D92
:204E000088F809102168C1F30721895D88F80A102168C1F30741895D88F80B102168090E6E
:204E2000895D88F80C10ADB2002DDCD1802804BF08F1280003F0D5F8802808BF03F04FF8C2
:204E4000802804BF06F2181003F0CBF8802804BF06F2201003F0C5F8802805D108F1100146
:204E600006F2101003F0CAF8802885D198F81010C9077FF581AF06F26C1003F0B2F80C2006
:204E80007AE700BFFC5D0000000C01402DE9F04182B005460C4605F00306FFF78DF9DFF8E5
:204EA000C47B97F82010012917D1802807D1F00004FA00F1284603F02EFDFFF717F9802849
:204EC0005DD100A92846FFF7BDFE802857D19DF80010A14253D00D2051E0DFF8A880F844C8
:204EE00008F1A208E9B211F808107970C5F3072111F80810B970C5F3074111F80810F970B6
:204F0000290E11F808103971F11914F808204A72802808BF02F0E5FF802804BF384603F074
:204F200060F8802804BF07F1080003F05AF8802804BF07F1280003F054F8802808BF02F03E
:204F4000CEFF802804BF08F2181003F04AF8802804BF08F2201003F044F8802805D107F188
:204F6000100108F2101003F049F88028A7D1397CC907A4D508F26C1003F033F80C20BDE84F
:204F8000F68100BFFC5C000080B5FFF733F9802804D11449DFF8D00AFFF7BAF902BD10B574
:204FA0000C4618B12246A02106F024FF2146012005F010FE3021012005F099FDDFF8AC0A7F
:204FC00003210170DFF8A80A8168091B81600021017310BD341C0020E01B0020B81B0020E5
:204FE00040350020F0ED00E0FCFFFF1F0100004001000080010000C0002000E0FCED00E0FA
:205000000CED00E00100FA0503005FA005005FA0010003013C1B0020F0B585B000200490A7
:20502000DFF8504A2078012807D0022800F08380032841D004283FD037E0DFF83C5A287CAB
:20504000202805D0302803D03C2800F0C5846CE00020697CA32908BF0120DFF8086A86F89F
:2050600020000127A42908BF002796F82000012804D103F053FBFFF739F802E0384603F0C6
:20508000ABF8ADF80800BDF80800802804D100220021022005F066FC02202070287C20282C
:2050A00005D10121002005F018FA05B0F0BD022102A8FFF774FFF8E7DFF8BC59297C202980
:2050C00001D0302931D1697CA32904D1DFF89429012382F820300127A42908BF002704288D
:2050E00002D101F02AFE01E001F0E2FCDFF8740990F82000012804D103F010FBFEF7F6FF32
:2051000002E0384603F068F8ADF80800BDF80800802804D100220021022005F023FC02205A
:205120002070287C2028C2D1BBE7022005F0E8F900210120B7E7DFF84059287C411E412909
:20514000F3D8DFE811F0C500D100D700F3006C0193019C0272030802360264023503D10394
:205160008302B7010E0218041B0439044200420042004200420042004200420042004200D6
:205180000A020A027400B300430042004200420042004200420042004200420042004200B7
:2051A0004200420074004F00D7006C019301B701DF010E0264028302F30010044904F300F6
:2051C000140442004D046D047C04AEE704F1200104F11C00FFF73EFA042104F11C00FFF71D
:2051E000DEFE62E704F1200104F11C00FFF732FAADF8080080280CBF0120002005F088FB68
:20520000DFF8785802A80178297041786970042204F11C01281D06F057FD042204F1200196
:2052200005F1080006F050FD0C212846D7E7697CA32915D1DFF82C6896F8200058B902F021
:2052400005FC03F06BFAFEF751FFADF80800012086F820001CE003F061FAFEF747FF15E0CA
:205260000127A42908BF0027DFF8F86796F82000012808D103F092FA384602F0ADFFADF825
:2052800008000020E4E7384602F0A6FFADF80800BDF80800802804D100220021022005F0C5
:2052A00061FB287C20287FF402AFFAE60120FEF766FF02F0CBFBDFF8AC07002180F820101C
:2052C0000022012005F04EFB012020700146E9E603A8FFF7D1FA9DF80C00002814BF8120DD
:2052E0008020ADF80800E2E6FFF7B7FB8020ADF80800DCE6DFF86C0790F8200010B902F035
:2053000023FF03E003F00AFAFEF7F0FEADF80800287C03287FF4CBAE03A8FFF719FB9DF8FC
:205320000C00002814BF80208120DAE70421ADF80A10042804BF0021ADF80A10DFF82C6747
:20534000317800293FD13D2806D10120FFF7DEF9ADF80800882009E00020FFF7D7F9ADF878
:205360000800287C3A280CBF58205420A080287C04280CD0BDF8080080280CBF012000202B
:2053800005F0C6FA0222A02102A806F033FDBDF80A00C0F1400292B200F1A00189B2DFF809
:2053A000E00606F027FD4021012005F013FC3021012005F09CFB02203070A0884038A080E7
:2053C0004020608071E66088BDF80A104942DFF8B02680180818A288412A12D34022A021F2
:2053E00006F008FD4021012005F0F4FB3021012005F07DFB608840306080A0884038A08075
:2054000053E6A02106F0F6FCA188012005F0E2FB3021012005F06BFB0320307045E6DFF8FC
:20542000446606F12401687CFFF79AF8ADF8080080280CBF0120002005F06AFA287C0528AF
:2054400004BF042106F124003FF4C9AEDFF82C5602A80178297041786970042206F12401B6
:20546000281D06F031FC08212846B8E6DFF8F465A87CE97C40EA0120297D40EA0140697D94
:2054800040EA01607062697C706AFEF7BFFFADF8080080280CBF0120002005F039FABDF8FF
:2054A000080080283FF403AE287C06287FF4FFAD812016E7DFF8AC65687CA97C40EA01208D
:2054C000E97C40EA0140297D40EA01607062687DA97D40EA0120E97D40EA0140297E40EA01
:2054E00001606061716AFEF713FFADF8080080280CBF0120002005F00BFA287C06287FF408
:20550000D6ADF3E6DFF85C65687CA97C40EA0120E97C40EA0140297D40EA0160706204F17B
:205520001401706AFEF796FEADF8080080280CBF0120002005F0ECF9DFF8405502A8017829
:20554000297041786970042204F11401281D06F0BBFB082169E6FFF717FD8020ADF8080030
:20556000A5E5DFF80065A87CE97C40EA0120297D40EA0140697D40EA01607062A87E019086
:20558000E87D00906B7E2A7E716AA87DFFF78CF9ADF8080080280CBF0120002005F0B8F903
:2055A000287C102804BF8020ADF80800022102A87FE5DFF8D044DFF8AC6406F1240120467A
:2055C000FEF748FE706ADFF8C014084370622146706AFEF79DFE03A8FFF714FA9DF80C00CD
:2055E000002814BF80208120ADF8080006F124012046FEF72FFE706A20F00C00DFF88C14B1
:20560000084370622146706AFEF782FE4FE5DFF85464A87CE97C40EA0120297D40EA01400F
:20562000697D40EA01607062AA7D697C706AFFF767F9ADF8080080280CBF0120002005F095
:2056400067F9287C0B287FF432AD4FE6687CDFF81014794401F20A4151F820100020FEF724
:2056600057FEADF8080080280CBF0120002005F04FF9287C0E287FF41AAD802031E6DFF895
:20568000EC03007800286FD1687CA97C40EA0120E97C40EA0140297D40EA0160A061687D00
:2056A000A97D40EA012041F60101884228BF4FF4C050A08000206080A088ADF80A008020A5
:2056C000A06040F60106DFF8B45313E005F020F9608800F500606080BDF80A00A0F50060DD
:2056E000ADF80A00A068802804D1A760802F1CBF0498E0606188A06908184919BDF80A20B6
:20570000B24204AB09D34FF40072FFF7CFF90746802F0CBF01200020D8E79208FFF7C6F981
:205720000646802E0CBF0120002005F0F1F8A068802804D1A660802E1CBF0498E060A0886D
:2057400041286ED34022A021CC4806F053FB4021012005F03FFA3021012005F0C8F9C34841
:2057600002210170402047E66088C44D4019A288412A0ED34022A02106F03CFB402101206E
:2057800005F028FA3021012005F0B1F96088403032E6A02106F02EFBA188012005F01AFA3E
:2057A0003021012005F0A3F9B048032101707CE4687CA97C40EA0120E97C40EA0140297D2F
:2057C00040EA0160A061687DA97D40EA0120412828BF4020A0808020A0600027A74DA08834
:2057E000D0B17919A069FFF72DFA0646802E0CBF0120002005F08CF8A068802804D1A66066
:20580000802E1CBFA069E060A069401CA0617F1CFFB2A0888742E4D1A088012804BF022028
:20582000A080A288A0219548B4E7904E3078C8B9687CA97C40EA0120E97C40EA0140297D14
:2058400040EA0160A061687DA97D40EA0120A080012030704FF44051022005F05AF98020A7
:20586000A06022E4A069A2888949412A22D31022FFF742FA0646802E0CBF0120002005F05E
:2058800047F8A068802804D1A660802E1CBFA069E060A0694030A061A0884038A080744876
:2058A0008168403981604FF44051022005F031F9FFF7FBBB9208FFF71FFA0646802E0CBF76
:2058C0000120002005F024F8A068802804D1A660802E1CBFA069E06065488168A288891AB6
:2058E00081600121FFF7DEBB604E3078B8B9012030704FF44051022005F00BF9687CA97C96
:2059000040EA0120E97C40EA0140297D40EA0160A061687DA97D40EA0120A0809FE7002519
:205920005B4FA08801281BDB3978A069FFF7AEFA0646802E0CBF0120002004F0E9FFA06834
:20594000802804D1A660802E1CBFA069E060A069401CA0616D1CEDB27F1CA0888542E3DB1C
:205960000121FFF79FBB022104F1080037E40C2104F1080033E40121FFF794BB3B4E3078A1
:2059800068B9687CA97C40EA0120A080012030704FF44051022005F0BCF8002011E5A288D2
:2059A000412A06D3608840306080A2F14000A08079E70121FFF776BB2C48007800287FF448
:2059C000D3AE697CA87C41EA0020A080002161804128FFF426AFB5E6687CFEF7D0FB80E4FC
:2059E000204E96F82000012818D1687CA97C40EA0120ADF80A00E87C297D40EA0120697D3B
:205A000040EA0140A97D40EA01607062BDF80A10706A04F00EFAFEF769FB68E4202066E4C4
:205A2000104890F82000012804D104F03CFAFEF75DFB00E02020ADF80800FFF738BB0948EA
:205A400090F82000012802D104F072FA00E00020ADF80A0002210DF10A00FFF72ABB00BFCE
:205A6000C8650000181B002001005FA02437002048370020E036002004370020341C00208B
:205A800040350020F0ED00E008005FA000005FA0C4350020DFF8A00C02497944891DC1663D
:205AA000704700BF450300002DE9F843DFF88C8C404605F0BFFCDFF8884C01202060DFF88F
:205AC000785CDFF8000D286405F1080068640020A8640A20E86400202865802068654FF4B9
:205AE0008077AF654FF48066EE65002028666866A86605F14001404605F0DAFC01220C21BD
:205B0000404605F0F9FCDFF8C08C404605F092FC4FF480302060DFF8B40C286405F2E0007C
:205B200068641020A8640120E864002028656865AF65EE65202028664FF40059C5F86490F4
:205B40000020A86605F14001404605F0B1FC01220821404605F0D0FC0121404605F0C3FCC9
:205B6000DFF86C8C404605F065FC4FF080702060DFF8740D2864002068641020A86400209F
:205B8000E864286580206865AF65EE6500202866C5F86490A86605F14001404605F088FCB5
:205BA000012208214046BDE8F84305F0A5BC00002DE9F04184B00121052005F011FD0121F6
:205BC000012005F004FD0121102005F000FD0121084605F0F3FC8020ADF8080004208DF820
:205BE0000B0003208DF80A00DFF8784C02A9204605F069FA4FF40070ADF8080004208DF8DB
:205C00000B0003208DF80A0002A9204605F05BFA2020ADF8080004208DF80B0003208DF823
:205C20000A0002A9204605F04EFA0121DFF8BC0C05F0BAFADFF8B85C4FF40041284605F0D0
:205C4000AAFA4021204605F0A6FA4FF4C06005F077FD0B208DF8000000208DF80100012001
:205C60008DF802008DF8030000A805F06EFD0F208DF8000000208DF8010001208DF802000B
:205C80008DF8030000A805F060FD11208DF8000000208DF8010001208DF802008DF80300F6
:205CA00000A805F052FD1E208DF8000000208DF8010002208DF8020001208DF8030000A895
:205CC00005F043FD06208DF8000001208DF801008DF802008DF8030000A805F036FDDFF887
:205CE000140C4FF480110160FFF7DEFE6FF00108404606F0C6F841F2941006F0BFF8002037
:205D000006F0BFF8012006F0CAF84FF0804005F071F8DFF8B47C384605F06CF8DFF8AC6CD3
:205D20004FF6FF703080112070800020706031464FF0804005F081F8002070803146384605
:205D400005F07BF84FF0804008210180002101834FF4A04181834FF48051018400203880F4
:205D600042F2221038834FF40450B88364203881002038844FF40060ADF804001C208DF80A
:205D8000070003208DF8060001A9204605F09BF94020ADF8040014208DF8070003208DF844
:205DA000060001A9204605F08EF94FF40040ADF8040010208DF8070002208DF8060001A912
:205DC000284605F080F9404606F05BF8DFF86809044979440E31C1660021417104B0BDE834
:205DE000F08100BF050000007047000010B504F06BFE0021012003F009FBDFF83C4901F00F
:205E000052FD08B90920B7E300F0C2FE08B91020F9E7DFF8780C00F06FFD002020710120A5
:205E200060714FF0804000210180172101854FF4405181830021018246F66A518186DFF8E1
:205E4000881B00220A800A840A8282894EF6FF531A4082818A8922F400728A81DFF87029C5
:205E6000136823F0010313601223536004F28003D360136843F001031360828942F4905241
:205E80008281112282828A8942F010028A810A8842F001020A80018841F009010180024886
:205EA0007844001DE06610BD0500000000F006BC10B504F009FEDFF88048218D012003F01E
:205EC000A5FA41F2941000F017FD00202071012060710020A08404F1A40000F07BFCA07948
:205EE000005D00F0FBFB02487844001DE06610BD05000000DFF840080179012911D1018FEF
:205F0000828C914203D20749794418316EE0816FC26F8267C167044979440C31C166002166
:205F2000017170478DFFFFFF0500000010B541F2941000F0E1FC00F005FCDFF8FC47A0791C
:205F400028B1001910F8010C00F0C8FB22E0E071DFF8740A018821F001010180818921F4A3
:205F600000718181DFF8D4170A6822F001020A600E224A6004F10802CA600A6842F0010251
:205F80000A6081894FF4007211438181018841F00101018002487844801DE06610BD00BFD0
:205FA00005000000DFF890070179012919D1018F828C914203D20B497944283116E0816F4A
:205FC000C26F8267C167817929B1064A7A441432491E817102E0044A7A440C32C266002189
:205FE0000171704749FFFFFF15000000C1660021017105214171062005F0EDBBDFF83807B2
:020000040800F2
:2060000002497944891DC166704700BFC10100002DE9F0410146002200230A70DFF81847F0
:2060200022816079658915B90128FBD0CAE0258F6089854238BF0720C0F0C4806281607958
:20604000A68916B90128FBD0BCE0A089A84238BF8023A2816079E68916B90128FBD0B1E046
:20606000E089A84238BF43F04003E2816079268A16B90128FBD0A5E0208AA8423CBF43F06A
:206080002003DBB222826079668A16B90128FBD098E0608AA8423CBF43F01003DBB2628222
:2060A0006079A68A16B90128FBD08BE0A08AA8423CBF43F00803DBB2A2826079E68A16B993
:2060C0000128FBD07EE0E08AA8423CBF43F00403DBB2E2826079268B16B90128FBD071E056
:2060E000208BA8423CBF43F00203DBB222836079668B16B90128FBD064E0608BA8423CBF05
:2061000043F00103DBB262830B706079A18B11B90128FBD056E0A08BA84238BF0122002013
:20612000A0834FF080452880DFF8BC6701203080254878449230185C904207BFA78F4FF059
:206140000108678F4FF006080020E071DFF87808018821F001010180818921F4007181817C
:20616000DFF8641A0A6822F001020A600E224A6004F10802CA600A6842F001020A608189BB
:206180004FF4007211438181018841F00101018041F2941000F0B0FB05F016FB0120A882F4
:2061A000288840F00900288000BF00BF378005F00DFB20890028FCD06079012802D100208A
:2061C00028804046BDE8F0817854000010B5DFF86845E07901285BD1208D216F4018FFF72D
:2061E00017FF012804D0062815D007281AD01CE0208D411C218589B2012003F007F9E08CF9
:20620000218D814213D14FF08040002101804FF4A0418183E8E11F4878447830E066062060
:20622000607103E06071062000E00620A6E188423EBF0D2060710620F8D37F20014203D0BB
:20624000144878444E3022E04FF08040002101804FF4A041818341F2941000F04DFBE08C62
:20626000218D401A80B20321A171E0708128A4BF8020E070606F80306067C0F30741A17010
:20628000C0F3072161702070034878440A30E06610BD00BF69FDFFFF19FCFFFF10B504F07F
:2062A00013FCDFF89444218D012003F0AFF841F2941000F021FB002020710120607104F13C
:2062C000B80000F087FAA079005D00F007FA02487844001DE06610BD0500000010B5DFF857
:2062E00058442079012820D1208FA18C884206D2002020710D4878443230E0663BE1A06F3C
:20630000E16FA167E0670020207141F2941000F0F3FA00F017FAA079001910F8010C00F041
:20632000DDF9034878440830E06610BD71FFFFFF3D00000010B541F2941000F0DDFA00F037
:2063400001FADFF8F443A07918B1001910F8010C02E0208D216F405C00F0C0F902487844BA
:20636000801DE06610BD00BF0500000010B5DFF8C8432079012831D1208FA18C884203D2C3
:20638000174878445A30F3E0A06FE16FA167E06741F2941000F0B0FA00F0D4F9A07988B157
:2063A000104979443E31E166401EA071C0B228B1001910F8010C00F091F90DE0208D216F85
:2063C000405CF8E7208D216F4018407800F086F9054878441230E0660020207110BD00BFB8
:2063E00055FFFFFF89FFFFFF3100000010B541F2941000F081FA00F0A5F9CF4C208D216FA7
:206400004018407800F06AF902487844801DE06610BD00BF0500000010B5C74C2079012805
:206420005DD1208FA18C884207D22D487844B030E0660020207105209EE0A06FE16FA1679D
:20644000E067208D411C218589B2012002F0DEFF00202071E08C218D814207D14FF08041B4
:20646000002008804FF4A0408883BDE0884238BF0D20E1D341F294107F2211420DD000F06F
:206480003BFA00F05FF9208D216F4018407800F025F9144878444C3020E04FF0804100226E
:2064A0000A804FF4A0428A8300F026FAE08C218D401A80B20321A171E0708128A4BF802038
:2064C000E070606F80306067C0F30741A170C0F3072161702070044878440C30E06610BD87
:2064E0000DFFFFFF35FFFFFFB5FDFFFF10B504F0EBFA0021012002F089FF41F2941000F08F
:20650000FBF98D4C002020710120607104F1CC0000F060F902487844801DE06610BD00BF8C
:206520000500000010B5844C207901281BD1208FA18C884203D20C4878442C3018E04FF0F5
:206540008040002101804FF4A04181836FF0010005F097FC054878441230E0660020607147
:20656000002102F053FF10BD85FFFFFF7DF8FFFFE06600202071052060710620BDE81040EC
:2065800005F029B910B56C4CE08F16214143C911A18513214143C911218600EB4001C9113E
:2065A000A18600EB80025200D2116285C0EBC000C011E0856186002000F056F94FF0804045
:2065C000002101804FF4A04181836FF0010005F058FC044878440C30E066002060710021AC
:2065E00010E000BF05F8FFFF6FF0010005F049FC01487844801C01E0F1F7FFFFE066002089
:206600006071218DBDE8104002F000BF38B504F05BFA0021012002F0F9FE41F2941000F02D
:206620006BF9454800210171C17101214171DFF89C151E220A80C28F1E324A804FF0804212
:206640000023138013854FF440539383002313824B885B1D9386DC4B00241C801C841C82BF
:2066600094894EF6FF552C4094819C8924F400749C81574C256825F001052560022565605A
:20668000E160216841F001012160918941F49051918111219182998941F0100199811988D6
:2066A00041F001011980118841F00901118002497944091DC16631BD050000001E48017981
:2066C000012907D1818CC1870021017102497944891DC166704700BFADFEFFFFF0B51649D8
:2066E000CA8E1446134D7D444A35465DCD6F012725F8027B4F8F25F8027B25F8022B4FF0A6
:20670000080C030646BFB1F83CE0A64407EB040E25F802EB131925F8023B40001419BCF1FA
:20672000010CEED1002E1ABF888F001938192880F0BD00BF0C4F00001C19002008000240F7
:206740000400024010B44FF08040DFF88414CA8E02EBC2024B8F9A18521D82869A4A0023AE
:2067600013801384138283894EF6FF5423408381938923F400739381154B1C6824F0010499
:206780001C6014245C60896FD960196841F001011960818941F490518181DFF838144FF4A3
:2067A00080130B6011218182918941F010019181118841F001011180018841F00901018096
:2067C00010BC70473408004058000240200800408000024010B44FF0804100220A800A85F7
:2067E0004FF440528A8300220A82DFF8E423D38E528F02EB8302521D8A86734A0023138085
:20680000138413828B894EF6FF5423408B81938923F400739381DFF8C0331C6824F0010411
:206820001C600A245C60D860186840F001001860888940F490508881DFF898034FF480131B
:206840000360908940F01000908111208882108840F001001080088840F00900088010BCBA
:2068600070470000000C0140F0B4D949012804D1488D4208CB8D4C8E03E0888D42080B8E24
:206880008C8E8C874B870A87C8860020CA8E4B8F8C8F012804BF182501F2A40607D00228E6
:2068A00007BF282501F2B806002501F2CC06012726F8027B5FEA056C36F802CC4CBFA444BE
:2068C0009C44A6F800C0052F3CBF02FB07FCA6F802C0361D6D007F1C062FEBD3401C032816
:2068E000D7DBF0BC7047000040000040000218000010014020ED00E010B504466FF001003C
:2069000005F0BFFA204605F0B9FA002005F0B9FA0120BDE8104005F0B4BA000070B5AC4C5D
:206920000020A084AD484FF4801101606579042D0CD0052D28D0062D31D0072D38D0092D2E
:206940003BD00B2D3BD0102D34D038E00426258D062004F043FF1C48002101804FF0804053
:2069600001804FF4A04181836FF0010005F089FA144878444E30E0660020607129463046E4
:20698000BDE8704002F042BD95480188022904D2491C01800120607170BD0526D7E7904884
:2069A0004188022902D2491C4180F3E70626CEE70726CCE710260025CAE70926FBE70A2601
:2069C000C6E700BF25F4FFFF000800406437002080B58448016809010ED54FF00061416099
:2069E0008148002101804FF08040018078480B214171062004F0EFFE01BD80B579480168EA
:206A000009030ED54FF4002141607748002101804FF0804001806E480B214171062004F0F3
:206A2000DAFE01BD10B56F4C206800070DD5082060606D48002101804FF080400180644864
:206A40000B214171062004F0C6FE2068400704D5042060605E480121C17110BD63485C49D7
:206A6000828E8A84028822F01002028001220A714FF0804100220A80818A21F4805181828A
:206A800056484FF4801101607047000020BF020080B56FF0010005F0F4F9002005F0F1F915
:206AA0004B48042141710620BDE8024004F093BE1CB50B208DF8000000208DF80100ADF84E
:206AC000020000A804F041FE0F208DF8000000A804F03BFE0B208DF8000000A804F035FED1
:206AE0001E208DF8000000A804F02FFE06208DF8000000A804F029FE4020ADF8040004206F
:206B00008DF807003A4C01A9204604F0DCFA4FF40060ADF8040001A9204604F0D4FA4FF428
:206B20000040ADF8040001A9324804F0CCFA4FF0804004F05FF92C4804F05CF904F0B8FAE0
:206B4000214804F077FC2C4804F074FC224804F071FC0021052004F043FD0021012004F012
:206B600036FD0021012004F029FD6FF0010005F088F9002005F085F91548044979440C3179
:206B8000C16600218180C17113BD00BF5DF2FFFF70B514240025164E002000BF401C302825
:206BA000FBD18021304604F0EEFA012804D16D1CEDB2052D01D370BD00252046441EC0B25E
:206BC0000028E9D170BD000008000240081C00201C19002080E100E08000024000E100E0FF
:206BE0007C37002000000240000800400C080040000C0140001001405800024080B5012155
:206C000044F2010004F0E3FC01210120BDE8044004F0E6BC10B582B04FF48060ADF80000E9
:206C200004208DF80300DFF8284B00A9204604F04AFA4FF40070ADF8000003208DF8020015
:206C400018208DF8030000A9204604F03CFA0220ADF8000003208DF8020004208DF803001E
:206C600000A9DFF8F00A04F02EFA13BD10B584B0DFF8E44A204604F077F9DFF8E00A40687D
:206C800000904FF48050ADF804000020ADF806004FF48060ADF808000020ADF80C000C2010
:206CA000ADF80A0000A9204604F0A0F90121204604F0E8F904B010BD00B585B04FF08040C2
:206CC00004F098F84FF6FF70ADF800000020ADF80200019000A94FF0804004F0AEF801221A
:206CE00040F60F614FF0804004F01EF90020ADF8080042F21070ADF80C0002A94FF0804008
:206D000004F0A8F800214FF0804004F017F901214FF0804004F019F905B000BD80B5FFF7F7
:206D20006DFFFFF777FFDFF8340A4FF461314160FFF79CFFBDE80140BEE710B582B04FF49A
:206D40008060ADF8000001208DF8020004208DF80300DFF8FC4900A9204604F0B4F94FF44B
:206D60000070ADF8000000A9204604F0ACF90220ADF8000000A9DFF8DC0904F0A4F9DFF8C2
:206D8000D80904F0F1F84FF0804004F033F8002144F2010004F01BFC0021012004F020FC62
:206DA00013BDF0B400204FF080410A8842F001020A80DFF8AC2913689BB19468DFF89839D7
:206DC00015686D1E156026789E801E88360602D40E8AB607F9D50E8A641CB60708D4002DC1
:206DE000EED14FF0FF3414600025DFF86C3914E0052016E0761E56601E88B60602D51E8815
:206E0000760602D40E8AB607F6D50E8AB607EFD4D6689F88AF556D1CADB25668002EE9D1F1
:206E200054600A8840F2FE331A400A808A8A42F001028A824FF6FD720A82F0BC704730B4E9
:206E400000204FF080410A8842F001020A800023DFF8042904E09BB2E46895881D555B1C17
:206E6000DFF8FC4865687DB16D1E65601588AD0602D515886D0602D40D8AAD07F6D50D8AF2
:206E8000AD07E8D5052002E04FF0FF3262600A8840F2FE331A400A808A8A42F001028A821A
:206EA0004FF6FD720A8230BC704710B5DFF8B008012101604160DFF8AC487F212170846097
:206EC000C460FFF76EFF052804D0207879280CBF00200120207010BD38B5DFF884480220D6
:206EE000206001206060DFF87C5800202870FF206870A560E560FFF754FF052801D1052020
:206F00001CE02878792818BF012017D101206060E560FFF794FF0528F1D028786870801CA3
:206F20006060A81CE060FFF78AFF0528E7D068784019C07879280CBF00200420287031BD83
:206F400038B5DFF81C480220206001206060DFF814582870FE206870A560E560FFF721FF55
:206F6000052801D1052013E02878792818BF01200ED10220687004206060A81CE060FFF70A
:206F80005EFF0528EED06879792814BF04200020287031BD38B5DFF8C847022020600120F4
:206FA0006060DFF8C05702202870FD206870A560E560FFF7F6FE052801D105201CE0287880
:206FC000792818BF012017D101206060E560FFF736FF0528F1D028786870801C6060A81C59
:206FE000E060FFF72CFF0528E7D068784019C07879280CBF00200420287031BDF8B50646AC
:207000000C46DFF85C570220286001206860DFF8547711203870EE207870AF60EF60FFF73C
:20702000C0FE052840D03878792818BF01203BD10520286001206860300E3870C6F3074084
:207040007870C6F30720B870FE70387879784840B9784840F97848403871AF60EF60FFF7FA
:20706000A0FE052820D03878792818BF02201BD102202860012068603C70E0437870AF60C6
:20708000EF60FFF78EFE05280ED03878792818BF032009D17C70601C6860B81CE860FFF7AD
:2070A000CEFE052818BF00203870F1BD70B50446DFF8AC560220286001206860DFF8A466CE
:2070C00021203070DE207070AE60EE60FFF769FE052801D1052024E03078792818BF0120CF
:2070E0001FD10520286001206860200E3070C4F307407070C4F30720B070F470307871786B
:207100004840B1784840F17848403071AE60EE60FFF747FE0528DDD03078792814BF0420F3
:207120000020307070BD2DE9F84381460C4690460025DFF82C660220306001207060DFF81A
:20714000247631203870CE207870B760F760FFF728FE052801D1052045E03878792818BFCB
:20716000012040D105203060012070604FEA19603870C9F307407870C9F30720B87087F868
:207180000390387879784840B9784840F97848403871B760F760FFF704FE0528DBD03878EA
:2071A000792818BF02201ED1781C621C98F800305D4018F8013B00F8013B521EF6D13C7074
:2071C000E01922466A408270E01C306001207060B760F760FFF7E5FD0528BCD038787928E5
:2071E00014BF042000203870BDE8F1832DE9F041074688461646DFF86845022020600120B2
:207200006060DFF8605543202870BC206870A560E560FFF7C6FD052801D105202EE028789E
:20722000792818BF012029D13EB1012E19D1FF20287000206870022012E02F7038460021B2
:207240006A1C7B1C98F8006002F8016B18F801CB8CEA0000491C9942F4DB49194870F81C2C
:20726000206001206060E560A560FFF79AFD0528D3D02878792814BF042000202870BDE871
:20728000F081F8B506460D46DFF8D4440220206001206060DFF8CC74632038709C207870D9
:2072A000A760E760FFF77DFD052801D1052025E03878792818BF012020D13E703046002168
:2072C0007A1C731C95F800C002F801CB15F801CB8CEA0000491C9942F4DBC9194870F01C72
:2072E000206001206060E760A760FFF75AFD0528DCD03878792814BF042000203870F1BDFB
:2073000038B5DFF85C540220286001206860DFF85444732020708C206070AC60EC60FFF70A
:2073200040FD052801D1052010E02078792818BF01200BD101206860EC60FFF780FD05281A
:20734000F1D0207879280CBF00200420207031BD38B5DFF80C540220286001206860DFF818
:207360000444822020707D206070AC60EC60FFF718FD052801D1052010E02078792818BF9F
:2073800001200BD101206860EC60FFF758FD0528F1D0207879280CBF00200420207031BDBC
:2073A00038B5DFF8BC530220286001206860DFF8B443922020706D206070AC60EC60FFF7AC
:2073C000F0FC052801D1052010E02078792818BF01200BD101206860EC60FFF730FD05281B
:2073E000F1D0207879280CBF00200420207031BD70B582B04FF6FF7425460220ADF80000C5
:2074000003208DF8020010208DF80300D14E00A9304603F058FE0221304603F0BEFE6519BD
:20742000ADB2002DFBD10221304603F0B4FE2046201880B20028FBD10220ADF80000032008
:207440008DF8020004208DF8030000A9304603F03AFE73BDF8B5C44D2878012806D00228F8
:2074600012D003281BD0042824D0F1BDBF48007C20B9FFF753FC0420287064E1022003F08F
:207480003FF80021012060E1B848007C0028F5D100F0DCFAFFF742FC0420287053E1B348E3
:2074A000007C0028EAD1FFF703FBFFF737FC0420287048E1AD4C207C102800F24881DFE81C
:2074C00010F042011E00230032003B004E005100A800B700F10015012F0132013B01170000
:2074E0003E011100FFF784FFFFF7C0FBFFF7DDFC0222A0219B4804F07DFC022124E0FFF7F1
:207500001CFC012028701EE1607CA17C090441EA0060E17C40EA0120217D08438F494860F9
:20752000FFF7A4FB0FE1FFF7D7FC4022A0218D4804F060FC402107E0FFF702FD0522A02190
:20754000884804F057FC0521012003F043FB3021012003F0CCFA864803210170F1BDFFF76A
:2075600019FDE2E77D4D824E7E4F307800283AD1A07CE17C227D637C42EA012141EA00403A
:2075800040EA0360A860617D298000226A80FFF735FD2888C21C2A8092B2412A14D340226B
:2075A000A021384604F026FC4021012003F012FB3021012003F09BFA0220307040206880F0
:2075C000288840382880F1BDA021384604F012FC2988012003F0FEFA3021012003F087FA49
:2075E00003203070F1BD6888C0192A88412A0ED34022A02104F0FEFB4021012003F0EAFAEA
:207600003021012003F073FA68884030D7E7A021DCE7A07CE17C227D637C42EA012141EA86
:20762000004040EA03604D4DA860FFF73FFD5FE74A4D4F4E3078C0B9207DE17C40EA0120C9
:20764000A17C40EA0140617C40EA0160A860607D401C288001203070002068804FF44051B4
:207660000220BDE8F44003F054BA2A88412A0CD340224049688840190C3004F025FB2888DE
:207680004038288068884030E7E73A49688840190C3004F019FB05F10C02617DA868FFF7A4
:2076A00042FD50E02D4D324E307878B9637C2B80FF2B04D101220021FFF798FD43E00120EC
:2076C000307000206880581C2880C7E72A88412ACED22849688840190C3004F0F5FA002280
:2076E00005F10C01607CFFF781FD2CE01B4D204E307830B9607C401C288001203070002003
:20770000ABE72A88412AB3D21A49688840190C3004F0DAFA05F10C01607CFFF7B2FD12E00F
:20772000FFF7EEFDE4E6FFF713FE0222A0210D4804F060FB022107E7FFF732FED8E6FFF723
:2077400057FEFFF793FA0121002002F0C6FEF1BD00080140000C0140003801403434002014
:2077600038370020341C0020E03600200437002024370020C435002010B586B0002000903A
:2077800001208DF8040000208DF805004FF4602002900020039001208DF81000DFF8984A1E
:2077A00000A9204603F01EFD012003F09CFD012301221121204603F059FD0121204603F05C
:2077C0002FFD204603F035FD204603F037FD0028FAD1204603F036FD204603F038FD002830
:2077E000FAD10121204603F038FD0221204603F08BFD0028F9D0204603F072FDDFF83C1A24
:207800000860012301220021204603F02FFD06B010BD10B5DFF8204A0121204603F01DFDF5
:207820000221204603F070FD0028F9D02046BDE8104003F055BD00B583B0DFF8000A0068DD
:207840000090FFF7E6FF0190082100A8FDF7A7FB03B000BD30B583B0DFF8E4492068C006EB
:2078600003D4206840F0100020604FF4C040ADF8000048208DF8030003208DF80200DFF890
:20788000C45900A9284603F01EFCA868C0F341300190206820F010002060042101A8FDF7F8
:2078A0007EFB03B030BD80B5FFF7B3FF40F2014188428041C043C00F02BD80B5062003F0F4
:2078C000AAFE4FF48070ADF8000018208DF8030003208DF8020000A9DFF86C09B0E3000036
:2078E00010B5DFF86809DFF86819086008210172DFF86049DFF860190C60DFF86019DFF8BC
:2079000060290A60DFF85C194FF400720A60DFF858194FF480120A60DFF850194FF400629D
:207920000A6001218172DFF848194FF404420A80244979448E31C97941722021002003F04B
:207940003AF994F82C10002003F04BF96021002003F030F9A021012003F02CF9E0210220FB
:2079600003F029F994F82C10022003F03AF94FF48071032003F01EF9DFF8F8080521017013
:20798000DFF8F408DFF8F4180160DFF8F40801210170002002F0A1FDDFF8E8080021017061
:2079A00001214FF4037003F012FEFFF7E5FE02F0B5FF00220021084602F0D4FFBDE8104022
:2079C0007BE700BFC045000010B5B6B01E4C7C44763430A82146112204F083F904A804F1FF
:2079E0001401B02204F07DF90020DFF89C482146DFF89828135C01F8013B401C0428F9DB5D
:207A00000420211DDFF88828135C01F8013B401C1028F9DB04A930A802F006FB04AA00A9A2
:207A2000204602F038FBDFF86C0800A9102211F8013B10F8014BA34218BF002002D1521EDD
:207A4000F5D1012036B010BDD83D000038B5DFF848080078012803D1BDE8314000F09EBE8C
:207A600002F01FFEDFF834480021204604F09CF8DFF82C580021284604F096F800212046A2
:207A800004F081F80021284604F07DF8204604F041F8284604F03EF800220221204604F0B7
:207AA0007BF800220221284604F076F800220121204604F071F8DFF8EC0703F0BBFCDFF8EC
:207AC000E80703F0B7FCDFF8E40703F0B3FC0021012003F073FD00214FF4805003F077FD6D
:207AE00000214FF4804003F07BFD00211020BDE8344003F06CBD2DE9F04186B00020ADF82F
:207B000000004FF48270ADF8020000200190ADF808004FF40070ADF80A002020ADF80C00D8
:207B20000020ADF80E000720ADF81000DFF86C4700A9204604F010F84FF44040ADF8000099
:207B40000020ADF80200DFF8585700A9284604F003F80121204604F027F8DFF8488740460B
:207B600003F068FCDFF84817DFF848770F60DFF8486706F28800486000208860706EC860B7
:207B8000002008618020486100208861C86108624FF40050486200208862404603F088FC33
:207BA000DFF80487404603F045FCF76006F27C00306110207061706EB0610020F06180204C
:207BC000306200207062B062F0623063706306F10C01404603F06CFCDFF8D076384603F0E4
:207BE00029FCDFF8D806B06306F29400F06310203064706E70640020B0648020F0640020FB
:207C000030657065B0654FF48050F0650020306606F13801384603F04BFC01220221204633
:207C200003F0BAFF01220221284603F0B5FF01220121204603F0B0FF0121204603F0A3FFD3
:207C40000121284603F09FFF06B0BDE8F08170B40020DFF86C164A684FF6FF7300E0401CF5
:207C60001488240601D59842F9D3984201D3022019E0002000E0401C14880CB99842FAD395
:207C80009842F4D200200C78DFF8285601E0401C2C881688F60701D59842F8D30C709842EE
:207CA0002CBF0220802070BC704710B5DFF8EC4500220221204603F06FFF00220221DFF83F
:207CC000E00503F069FF00220121204603F064FF0021DFF8D40503F006FC0021DFF8CC05D5
:207CE00003F001FC0021DFF8BC0503F0FCFBDFF8D40503F00DFC802010BD2DE9F041054646
:207D00000E468024002716B1012E18BF062402F0DBFE802C02D1FFF79AFF0446802C08D1A5
:207D20000021DFF8940500EB8600C06E00F08AF80446802C02D1FFF78AFF0446802C0DD185
:207D40004FF6FF7800E07F1C4FF4007003F0DFFB08B94745F7D3474528BF0324802C0ED130
:207D600000274FF6FF7800E07F1C4FF4003003F0CEFB08B94745F7D3474528BF0324802C19
:207D800002D1FFF792FF0446802C54D1DFF8287506207866B86107F2A0003861DFF8088547
:207DA00007F10C01404603F083FB0620786406EB460007EB400000F2A800F863DFF8EC6440
:207DC00007F13801304603F073FBDFF8E4140620C8604D60DFF8CC54284603F069FB0121F3
:207DE000304603F080FB0121284603F07CFB0121404603F078FB01220221DFF8A40403F0DF
:207E0000CBFEDFF8985401220121284603F0C4FE01220221284603F0BFFE00274FF6FF752A
:207E200000E07F1C202003F072FB08B9AF42F8D3AF4228BF0324802C0CBF0120002002F001
:207E400067FDCBE0F8B506460F46002E01D10620F2BDFFF72AFF0446802C3ED1DFF8585449
:207E60005FB10120696E022907D34119097907F8011B401C696E8842F7D302206866A8613E
:207E80002E61DFF8246405F10C01304603F010FB02206864A86EE863DFF8107405F13801A4
:207EA000384603F005FB0121384603F01CFB0121304603F018FB01220221DFF8E40303F012
:207EC0006BFEDFF8D85301220221284603F064FE01220121284603F05FFE2046F2BD0021F5
:207EE00002E0002104E00146DFF8DC03AAE70146DFF8D803A6E72DE9F04106460F46FFF7A9
:207F0000A6FE0446802C02D1FFF7CFFE0446802C64D1DFF8A4535FB10120696E022907D32B
:207F20004119097907F8011B401C696E8842F7D306206866A8612E61DFF86C6305F10C014E
:207F4000304603F0B5FA0620686405F2B400E863DFF8587305F13801384603F0A9FADFF865
:207F600050130620C860281D4860DFF83883404603F09EFA0121384603F0B5FA01214046D6
:207F800003F0B1FA0121304603F0ADFA01220221C34803F001FEC14E01220121304603F011
:207FA000FBFD01220221304603F0F6FD00264FF6FF7700E0761C202003F0A9FA08B9BE423D
:207FC000F8D3BE4228BF032408D2287900F00700022803D004280CBF072408242046BDE800
:207FE000F08138B50446642500212046FFF783FF6D1E072801D1002DF6D132BD70B5044673
:020000040800F2
:208000000D46642629462046FFF775FF761E072801D1002EF6D170BD80B5E020ADF80000B3
:2080200003208DF8020018208DF8030000A9864803F049F84FF46040ADF8000000A9A4480E
:2080400003F041F801BD38B49D4B5B681C88A40701D4022020E0994C208096480180002154
:208060004FF6FF7400E0491C1D88AD0701D4A142F9D3A142EDD2002100E0491C1D88ED0785
:2080800001D4A142F9D3A142E3D2002A008814BF10708DF80000802032BC704710B582B0FE
:2080A000854C002020700022FF21C020FFF7CBFF802848D10022FF210020FFF7C4FF8028D9
:2080C00041D100AA7F210020FFF7BDFF80283AD19DF80000002801D1052016BDFF2809D137
:2080E00020780830207000AAFF210020FFF7ABFF802828D19DF80000FF2823D0802021780D
:208100009DF8002002E0491CC005000E80EA0203FF2B01D00128F6DA2170002812D02078FA
:20812000082807D104F27600A06604F27A00E066802016BD092802BF04F27400A06604F244
:208140007800F4D0042016BD70B582B0534C00220221204603F020FD514D002202212846EA
:2081600003F01AFD00220121204603F015FDA0898DF80000524840680088800758BF022608
:2081800014D500220021FE20FFF75DFF0646802E02D1FFF783FF0646022E07D00022002168
:2081A000FE20FFF750FF802E08BFC6B201220221284603F0F1FC01220121204603F0ECFC55
:2081C00001220221204603F0E7FC802E02D1FCF729F80646304676BD10B504463D48772167
:2081E000017041708170C170017141710121012003F0E4F901214FF4805003F0E8F90121D9
:208200004FF4804003F0ECF90121182003F0DFF9204602F0D9F9FFF76EFCBDE8104093E765
:2082200080B517480078ADF80000022100A8FCF7B6FE01BD00000000002401406C37002035
:20824000181002400010014000080140B8360020D4360020481B0020D8360020DC360020FF
:20826000BC1A00205C3700205837002060370020843700208A3700200437002055534243AB
:20828000E0360020201C002028370020E0F7FF1FE4F7FF1F003C0008381B002000300140B7
:2082A000003800401C00024030000240580002403C3600200C300140001A00200C3800400F
:2082C000F01B002020020200101C0020121C0020000C0140341C002038B54FF40050ADF8D3
:2082E000000010208DF8030003208DF80200DFF8F45800A9284602F0E6FE4FF4A040ADF844
:20830000000004208DF8030000A9284602F0DBFE2020ADF8000004208DF8030003208DF896
:208320000200DFF8C44800A9204602F0CCFE1020ADF8000004208DF8030003208DF8020062
:2083400000A9284602F0BFFE1020ADF800008DF8030003208DF8020000A9204602F0B3FE9E
:2083600000221021204602F01AFF0220ADF8000010208DF8030003208DF8020000A9204601
:2083800002F0A1FE00220221204602F008FF31BD10B582B004208DF803004FF4E040ADF80F
:2083A000000000A9DFF83C0802F08DFE04208DF803001220ADF80000DFF82C4800A920469F
:2083C00002F081FE4FF48460ADF8000000A9204602F079FE13BDDFF81408016841F4005136
:2083E0000160416841F400514160704710B5DFF8FC07016841F4804101603524FFF7EBFFFD
:20840000641EFBD110BD0000F8B507460C460026DFF8DC5747FA06F0C00742BFE86840F442
:208420008040E86003D4286940F480402861FFF7D2FF761C082EEDDBDFF8B80702210160DE
:20844000286820F070602860286840F080602860002020700121EA6842F40052EA6000BF47
:2084600000BF00BF00BF00BF00BF00BF00BF00BF00BF00BF6A68D20404D5227801FA00F37D
:208480001A4322702A6942F400522A61401C0328E1DBF1BD2DE9F84380460D4600270024A1
:2084A000DFF84C67DFF850971BE0012F19DBFFF792FF00BF00BF00BF00BF00BF00BF00BF95
:2084C00000BF00BF00BF00BF0220C9F80000306820F070603060306840F040703060FFF7B7
:2084E0007AFF00A94046FFF78FFF781CC7B29DF80000022803D1042FD7DB012446E0012857
:2085000040D10020286001460122F36843F40053F36000BF00BF00BF00BF00BF00BF00BFC7
:2085200000BF00BF00BF00BF7368DB0407D52B6802FA01F73B432B6080F00100C0B233699A
:2085400043F400533361491C2029DEDB0021F26842F40052F26000BF00BF00BF00BF00BF86
:2085600000BF00BF00BF00BF00BF00BF7268D20448BF0121326942F400523261814205D05A
:20858000042403E004280CBF02240324FFF723FF00BF00BF00BF00BF00BF00BF00BF00BF7C
:2085A00000BF00BF00BF484602210160306820F070603060306840F040703060FFF70BFF5C
:2085C0002046BDE8F28300002DE9F04182B0064688460027DFF81856DFF81C4601E0042FCF
:2085E0004ADA00A93046FFF70FFFFFF7F4FE00BF00BF00BF00BF00BF00BF00BF00BF00BF95
:2086000000BF00BF02202060286820F070602860286840F040702860FFF7DDFE7F1CFFB22D
:208620009DF800000228DAD0012827D10027002628FA06F0C00707D5E86840F48040E8601C
:2086400087F00107FFB203E0286940F480402861FFF7C1FE761C202EEADB012F02BFE8685E
:2086600040F48040E86003D0286940F480402861FFF7B1FE002005E0012003E004280CBF38
:2086800002200320BDE8F68138B5044600200090DFF8685500A96878FFF7FCFE08B110308C
:2086A0000AE00099B222114207D004F01E01287BFFF78AFF08B1183080B232BD70B5044673
:2086C000DFF8340502210160DFF82455286820F070602860286840F040702860FFF786FE4C
:2086E000002644FA06F0C00742BFE86840F48040E86003D4286940F480402861FFF76BFE88
:20870000761C102EEDDBFFF771FE286940F480402861FFF760FEBDE870405CE610B582B06C
:2087200000200090DFF8D444DFF8D4042061FF2060610020A061E0612062FFF7CDFD01F0F5
:20874000DBFA4EF29E70FFF7B9FF04F118012078FFF7A0FE10B1083080B216BD1E20FFF7DC
:2087600093FF002819D14FF0A041607BFFF72CFF08B11830F0E700A96078FFF78BFE10B1A0
:20878000103080B216BD009800F0704010F1805F01D0302016BD00F013F816BD80B54EF245
:2087A0003C70FFF78BFFDFF85404DFF854140161FF214161FFF7ECFDBDE8014001F008BB82
:2087C00038B500200090F02000F027F8002823D1DFF8284400A9E079FFF75CFE050006D051
:2087E0001E20FFF751FF05F1200080B232BD04F11C01A079FFF74EFE0500F1D104F1200174
:20880000E078FFF747FE050005D01E20FFF73CFF05F11000E9E7002032BD70B50446002503
:20882000DFF8D8633069A04210D02146B07BFFF7CBFE050009D0DFF8C80330611E20FFF735
:2088400023FF05F1180080B270BD3461284670BD70B500240546DFF8A4637169A94225D02D
:20886000022807D1DFF89C430020FFF7D6FF00280CD070BD012808BFDFF88C43F4D00028A2
:2088800008BF4FF00C54EFD0382070BD2146307AFFF79AFE040008D0FF2070611E20FFF78F
:2088A000F3FE04F1280080B270BD7561204670BD70B582B004460D460020FFF7AEFF002803
:2088C00028D1DFF838632146707AFFF77DFE040006D01E20FFF7D8FE04F1280080B276BD05
:2088E00000A9F079FFF7D6FD040005D01E20FFF7CBFE04F12000F1E72946F078FFF7CAFD46
:20890000040006D01E20FFF7BFFE04F1100080B276BD002076BD70B582B004460D460020BB
:208920000090FFF77AFF002834D1B44E2146707AFFF74AFE040006D01E20FFF7A5FE04F1D4
:20894000280080B276BD2946F07AFFF73DFE0400F2D1AE48016841F480410160FFF73BFDD5
:20896000FFF739FD00A97078FFF794FD040001D01030E6E70098000601D52D2076BD009845
:20898000800601D52E2076BD0098800701D52F2076BD002076BDF8B504460D460020FFF7D0
:2089A0003CFF002833D1954E9949707AFFF70CFE070006D01E20FFF767FE07F1280080B2D9
:2089C000F2BD1020FFF729FF002820D104F07F01707AFFF7F9FD0700ECD12946B079FFF7E5
:2089E00059FD070005D01E20FFF74EFE07F12000E5E72946F078FFF74DFD070006D01E20AF
:208A0000FFF742FE07F1100080B2F2BD0020F2BDF8B504460D460020FFF7FFFE002822D1F0
:208A2000764E7B49707AFFF7CFFD070006D01E20FFF72AFE07F1280080B2F2BD1020FFF7A2
:208A4000ECFE00280FD12946B07AFFF7BDFD0700EDD104F07F0040F48031707AFFF7B4FD2D
:208A60000700E4D10020F2BD2DE9F04782B08046894692460027002418F00F0018BF4020E6
:208A80005FD10220FFF7E4FE0546002D5B4E02D0284656E0641C544552D2002D50D100206A
:208AA000FFF7BBFE0546002DF2D108EB8401707AFFF78AFD070006D01E20FFF7E5FD07F102
:208AC000280080B23DE01020FFF7A7FE0546002DDED100A93079FFF7DDFC0028DFD109EB40
:208AE00084017079FFF7D6FC070005D01E20FFF7CBFD07F12000E4E7641C544507D209EB9F
:208B00008401B079FFF7C6FC0700EFD1641C544507D209EB8401F079FFF7BCFC0700E5D1E9
:208B2000641C5445B7D209EB8401F078FFF7B2FC0700AFD01E20FFF7A7FD07F11000C0E701
:208B40003846BDE8F6872DE9F84F804689469246002718F00F0018BF402040D10220FFF70D
:208B600077FE05467DB1284639E0574507D259F827103078FFF728FD0446ACB97F1C761CE4
:208B8000BBF1010BF1D157451FD2F5B90020FFF744FE0546002DE6D1184E08EB8701707ACE
:208BA000FFF712FD044634B11E20FFF76DFD04F1280080B213E01020FFF72FFE0546002DD6
:208BC000D1D108364FF0040BD1E71048016841F480410160FFF7FFFBFFF7FDFB0020BDE8F4
:208BE000F28F0000000C014000080140100C0140040C01401008014014080140A01B00201F
:208C0000F00000FF0200002301000023140C0140F0ED00E010B5DFF8BC47002800D12FE057
:208C2000DFF8B40700680068804720680A3010BD80B5DFF8A0070068C178DFF8A0275278C0
:208C40008A420DD38278002A0AD18288002A07D18172DFF88407006840688047002002BD52
:208C6000022002BD10B5DFF86C47002800D107E0DFF8640700688068804720680C3010BDFA
:208C8000206801210182002010BD10B5DFF844472068C1784079DFF8482712689269904787
:208CA00021688A7A002A07D0002805D10879002802D18878002801D0022010BDDFF81807CE
:208CC0000068C068804720684179C1722068C1780173002010BD10B5DFF8F8160968002863
:208CE00003D102200882002010BDDFF8F8460020208008787F22104216D1487A810603D5B7
:208D0000002141F0020121704006207809D540F001002070DFF8C006006800698047204655
:208D200010BD00F0FE00F4E700F07F02012AF6D000F07F000228D6D1487900F00F01DFF863
:208D4000A826000652F8210005D500F030001028E0D10020DBE700F44050B0F5805FD9D15D
:208D60000020D4E770B5DFF86C060068017811F07F0102BF417A01F0DF01417254D00229F9
:208D800005D14188002902D10179002901D0022070BD417921F08005DFF84C460A0654F860
:208DA00025204CBF02F0300202F44052DFF82C361B789D42EBD2002AE9D0807A0028E6D094
:208DC000080654F825000BD500F03000102826D1284601F0D9FE3021284601F088FE1EE07B
:208DE00000F44050B0F5805F19D14BF68F7665B9DFF8F80590F82C10002001F0F2FE2068FC
:208E0000304080F44050206009E0284601F0ACFE54F82500304080F4405044F82500DFF84F
:208E2000B805006840698047002070BD38B5DFF8A4050268537923F08000DFF8AC151C0660
:208E400051F820404CBF04F0300404F44054DFF88C552D78A84207D25588002D04D1002C7F
:208E600002D0927A002A01D1022032BD1A0651F8202042BF48F6BF731A4082F0100204D437
:208E80004BF68F731A4082F4805241F82020DFF84805006880698047002032BD80B5DFF81D
:208EA00034050068417A41F020014172DFF828050068C0698047002002BDDFF81825126888
:208EC000538A20B98888C01A108200207047086818187047F8B5DFF8FC54286800F11004C9
:208EE0002688A168080015D0A6B1A088864288BF06463046884707462088801B2080608897
:208F000030186080002001F05EFE32460146384602F084FF208860B1DFF8D4044FF44051CE
:208F200001800021002001F055FEDFF8C8043021018028682188A288914202D30321017214
:208F4000F1BD002901D00521F9E706210172DFF8A804006880B2DFF8A414002241F8102092
:208F6000DFF8900430210180F1BD38B5DFF864442068457801787F2211422CD1092D02D1E2
:208F8000FFF756FE38E0052D0BD1C178802906D2817821B9818811B9807A002839D00820AE
:208FA00045E0032D0AD1C178012926D1818821BB407A800621D5FFF771FF1DE0012D1CD18E
:208FC000C178012919D18188B9B9407A800614D5FFF7C8FE10E001F07F00012804D10B2D4E
:208FE0000BD1FFF752FE07E0022806D1012DEFD0032D02D1FFF71AFF58B12846DFF8E01327
:20900000096849698847032808BF09200FD00028C5D10620DFF8E013096889B2DFF8DC2334
:20902000002342F81130DFF8CC1330220A802168087231BD2DE9F041DFF8984320684178D5
:2090400006291AD101787F22114239D18078012802BFDFF88C030068C16900F0818002288A
:2090600002BFDFF87C030068016A79D0032827D1DFF86C030068416A72E0002947D14188E5
:20908000F1B9C18802291BD10179C9B901787F22114206D1828822B96149794401F5C17112
:2090A0005EE001F07F02012A16D100214079CC4A12689269904718B92068807A0028EBD17B
:2090C00020684078C649096809698847032850D1206809210172A0E001F07F010229EFD142
:2090E000407900F00F0100F07002BF4B000653F821004CBF00F0300000F44050B74B1B7895
:209100009942DDD2002ADBD10028C5D1D8E7082908D100787F210842D2D14249794401F525
:2091200082711DE00A29CBD1017801F07F010129C6D1817A0029C3D041880029C0D1017911
:209140000029BDD1C1880129BAD100214079A44A1268926990470028B2D133497944C83169
:209160000800ADD0206800224282816100208847002021680A8A4FF6FF739A4202D109205F
:2091800008724AE0022800D00AB90820F8E7087800063CD5C888904238BF088290480068ED
:2091A00090F82C00888201F11005288828B9097A042904BF0726102024D0AF88874205D3BD
:2091C0000426B84288BF3846074600E00226B8B2A96888478046002001F0F4FC0146BAB28D
:2091E000404602F007FEB9B2002001F0F3FC2888C01B288068883818688030207C494FF4D4
:2092000040520A807B4908802068067205E00320087277484FF440510180BDE8F08100BF7B
:20922000B7FAFFFFF1F9FFFF3DFAFFFF38B574487149096889B2734A32F8111000EB41001F
:20924000644C21680A7A092A14D010F8012B0A70216810F8012B4A70851C35F8040B01F047
:2092600009FD21684880288801F004FD21688880A888C8802068012101722068C08810B936
:20928000FFF773FE01E0FFF7D5FEBDE831406FE02DE9F0414F4C2068017A022901D004294A
:2092A00034D100F11005288820B9042904BF0726102024D0AF88874205D30426B84288BF96
:2092C0003846074600E00226B8B2A96888478046002001F077FCBAB20146404602F08AFD75
:2092E000B9B2002001F076FC2888C01B288068883818688030203E494FF440520A803D4969
:209300000880206806722068007A14E0062911D1417805290AD101787F22114206D1C07880
:2093200000F040F82C480068006A80472C48006880688047082021680872BDE8F04117E075
:2093400010B5244C2068007A032801D0052804D1FFF7C0FD2068007A06E0072803D12048D2
:209360000068C0688047082021680872BDE8104080B51E4890F82C10002001F032FC15487B
:209380000068017A082906D119494FF480520A80184910220A80007A092801D1012002BD67
:2093A000002002BDF0B40D49097800220E4B59B11C4648F68F7526682E40D7B23E4344F8E8
:2093C000046B521C8A42F6D340F08000D864F0BC70470000D4360020DC3600200C1C002028
:2093E000D836002074370020005C0040481B00208037002082370020505C00400460004015
:2094000000600040086000407047000038B504460D4602F0D9F9DFF87404012C1CBF002187
:2094200001720473A0F80D50601E8041C00F01F06FFABDE8314002F0C9B901280CBF002047
:209440000220DFF84814087001204870DFF84004027812098A70407800F03F00C8707047E6
:2094600080B500B10120FDF7FFF900210020BDE80440CBE780B5042826D8DFE800F0151BD7
:2094800003090F00DFF80C04104979443E311AE04021DFF8040401F080FEE6E74021DFF897
:2094A000F80301F078FEF8E7DFF8E803084979441E3108E0DFF8E40300210180DFF8D40356
:2094C000044979440E31016001BD00BF41D1FFFF1DC9FFFF19D0FFFF10B4DFF8C0330024D8
:2094E0001C80DFF8BC3303241C70DFF8B83300241C80DFF8B4331880DFF8B033D8708128D4
:2095000024BF8020D870C1F307409870C1F3072058701970DFF898030160DFF898030260AA
:20952000DFF8700301497944891C29E071CDFFFF10B4DFF8683300241C80DFF87C331C80D8
:20954000D74B03241C70D74B00241C80D64B1880D64BD870812824BF8020D870C1F30740C3
:209560009870C1F3072058701970D1480160D1480260C84801497944891C01E035C9FFFF29
:20958000016010BC7047000070B582B04FF4C050ADF80000C94D2A7CBC4C207AC0EBC001CE
:2095A000B948784400F2E22000EB4100105C012805D1022000F0A4FF0021012060E1C04E1D
:2095C0003078012807D0022809D003280DD0042800F0448173BD002AEBD1002044E1002A72
:2095E000E7D1FEF733FA287C3EE10D2AE1D8DFE812F00F00160022003D00430049004F00B6
:2096000055005A0006016000CA00E2001E01D0E7227200220021022001F0A4F92EE1227288
:20962000FDF746FA00220021012001F09BF901203070014623E12272687CFFF7FEFE08226D
:20964000A021204602F0D6FB9E48032101709E48816808398160002101730821012001F0E4
:20966000B9FA3021012001F042FA73BD2272687CFFF7F6FE012102E122720020FFF7FAFE5F
:209680000121FCE022720120FFF7F4FE0121F6E022720220FFF7EEFE0121F0E02272FFF723
:2096A000E9FE0121EBE022720420FFF7E3FE0121E5E0844E3078002843D1687CA97C41EA76
:2096C00000202082297D6A7D120242EA0141AA7D1143A161A0820021E18241F60101884293
:2096E00004D300210820FFF791FE62E7092810D2024605F1170104F11C0002F0E5FA287C8D
:20970000207204F11C02A169A08AFFF7E5FE0121B5E0082205F1170104F11C0002F0D4FAD7
:2097200008206082208A083820826748816808398160012030704FF44051022001F0E9F94F
:2097400073BD608A0019228A6049412A0ED340221C3002F0B9FA608A40306082208A403884
:2097600020825948816840398160E4E71C3002F0ABFA287C207204F11C02A169A08AFFF742
:20978000ABFE01217BE0687CA97C41EA00202082297D6B7D1B0243EA0141AB7D1943A1610D
:2097A0000023E3826382A082227204F11C02FFF7BFFE012163E0608A0019A28A414E412A32
:2097C0000ED34022A0211C3002F014FB02203070608A40306082A08A4038A08240213DE7F1
:2097E000A0211C3002F006FBA18A012001F0F2F93021012001F07BF90320307068E0042239
:20980000A02104F10C0002F0F5FA2E48032101702D488168091F8160002101730421012058
:2098200001F0D8F93021012001F061F9E6E70222A02100A802F0DEFA22480321017022481C
:209840008168891E8160002101730221012001F0C1F93021012001F04AF939E0002A7FF4B7
:20986000A8AEFDF76AFA287C2072FCF7A1F900220021022001F076F80320307001210020AE
:2098800000F02BFE73BD00BF5C200000181C0020FE3F000888190020000C01407C370020CA
:2098A0002219002044190020421900201C190020901900208C1900207E3700200437002042
:2098C000E03600202437002048370020C4350020287C207273BD0000DFF88C032949794424
:2098E000A2310160284979449E314160274979449A318160264979449631C160254979447E
:2099000092310161244979448E314161234979448A318161224979448631C16121497944A9
:2099200082310162204979447E314162CF481F497944783101601E4A7A4474324260816004
:20994000C16001611B4A7A446A3242618161C1610162194979446031C164184979445C313B
:2099600041651749794458314162164979445431C1621549794450314163144979444C315D
:2099800041647047C9000000390100000F0200000D0200000D020000510200009302000051
:2099A00097020000990200009B0200005DFAFFFF690000008300000010270000C825000071
:2099C000A4270000E8250000A02600003427000010B4A748016842688068D9B1A54B99705D
:2099E000C1F307241C71C1F307449C71090E19729A72C2F307211973C2F307419973110EB0
:209A000019749874C0F307211975C0F307419975000E187610BC704780B597480068807AA6
:209A200040B1012001F0B0F8022001F09DF893480021017001BD80B591480068914988428E
:209A40001CBF022000F05CFD01BD000038B5FFF7BFFF894C20680021817202F067FA8A48CB
:209A6000002141604FF40441884A118001602068124979444631C97941721020ADF80000F7
:209A80008DF8030003208DF80200814D00A9284601F019FB2068807A38B91021284601F0A7
:209AA0007AFB2068807A0028F7D01021284601F074FB78480521017031BD00BFC8240000D1
:209AC00010B5754800218172002001F001F84FF40071002001F003F82021002001F007F8D5
:209AE0002021002001F067F85F4C94F82C10002001F077F86021002001F05CF8002001F0CB
:209B000027F8002001F01AF80021012000F0E7FFA021012001F04EF82021012000F0E7FF9A
:209B20000021012000F0F5FF0021022000F0D7FFE021022001F03FF894F82C10022001F0D0
:209B400050F84FF44051022000F0E3FF0021022000F0CDFF0021032000F0C1FF4FF48071CE
:209B6000032001F027F82021032000F0C0FF0021032000F0CEFF94F82C10002001F031F89C
:209B8000002000F0DBFF0020FFF70CFC3C483D4901603A480021017010BD70477047000003
:209BA00080B5354909680A7802F07F02212A0FD1FE280DD1488800280AD18888002807D17A
:209BC000C888012804D1074878441830020001D1022002BD88610020488200F03BF8002019
:209BE00002BD00BF7100000080B5234909680A7802F07F02212A18D1FF2816D14888002835
:209C000013D18888002810D1C88800280DD1012000F0BAFF022000F0A7FF1948194901604B
:209C2000164800210170002002BD022002BD01B900B1022070471949FFF73FB91849FFF789
:209C40003CB90D490968C978084A02EBC1012431FFF733B9002805D1074800680121018275
:209C6000002070470F487047481B0020BC1A0020E8F7FF1FC41B0020D436002024370020E5
:209C80000437002055534243405C004084370020001001408A370020B8360020081B002002
:209CA000101B00207837002010B586B0029000200390ADF81000ADF814000420ADF8120001
:209CC000002000904FF40070ADF804000020ADF80600CE4C204601F047F900A9204601F0FC
:209CE000C5F902A9204601F081F901224021204601F0D1F906B010BD30B58DB04FF48060BD
:209D0000ADF8040004208DF8070003208DF8060001A9BF4801F0D7F901214FF4804001F0B4
:209D200056FC0121012001F049FCBA4DA869FFF7BBFF00214FF4804001F049FCB64C2046CE
:209D400001F078FBB5484FF4803101604FF4805105F11C0002F000FAB1480290686905EBEF
:209D6000C02101F21C0103910021049105EB400080880590069180200790089109910A913F
:209D80004FF400500B900C9102A9204601F090FB01220221204601F0AFFB00220821204673
:209DA00001F0AAFB00220421204601F0A5FB0F208DF8000000208DF8010001208DF80200CD
:209DC0008DF8030000A801F0C0FC00200DB030BD1CB58E48818921F400518181018809072A
:209DE00044BF8188ADF8041001F0BEF88A4C204601F020FB00220221204601F07DFB0F206C
:209E00008DF8000000208DF8010001208DF8020000208DF8030000A801F097FC00214FF437
:209E2000804001F0D4FB0021012001F0C7FB002016BD70B504460E46764D2878012808D192
:209E4000A8884000B04202D1A869A04201D000F02AF841F20100864207D27008A880E8801A
:209E6000A869A0420DD0002C01D1382070BD01214FF4804001F0ABFB2046FFF715FFAC6156
:209E800004E001214FF4804001F0A1FB002028616861A8812881E888688102F00FF8012075
:209EA0002870002070BD80B55848818921F4005181810188090744BF8088ADF8000000210C
:209EC0004FF4804001F083FB0021534801F00BFB504800210170002002BD82B05148016820
:209EE000890323D5416841F4403141604748818921F4005181810188090744BF8088ADF8A4
:209F00000000444841694A4200EB42025389D288934209D1C1F10101416100EB41000021C8
:209F2000018102B001F0CABF0121417002B0704710B5384CE089002802D12078002801D1F8
:209F4000002010BD2069616988420AD1324801F0DBFA216904EB41018A88101A0989401AF9
:209F600004E004EB400081880089081AE08100F002F8E08910BD38B5264CE589C5B1412DE8
:209F800028BF402520692A464FF4807104EB40031B8904EBC02018181C3001F02BFFA581E6
:209FA000A189032000F016FE3021032000F09FFD31BD10B5174C206904EB4000A1890289CD
:209FC0008A180281E089401AE0810021A18180B208B1FFF7D0FF206904EB400001898088FB
:209FE000814212D3607801280BD1002060706069C0F10100606104EB40000021018101F0ED
:020000040800F2
:20A000005DFF2069C0F10100206110BD003801400008014000080020580002400400024091
:20A020000438014000000240F0B5046842688368C0680C604A608B60C860DFF8B4520A265D
:20A04000DFF8B072C0F3074C1CF807C0C0F3072E1EF807E04FEA0E4E4EEA0C6C5FFA80FE25
:20A060001EF807E04CEA0E2C4FEA106E1EF807E04EEA0C0C55F804EB8EEA0C0C8CEA040425
:20A0800062405340584041F8104F4A608B60C860761ED7D1F0BD2DE9F047036814686340DE
:20A0A000446855686C40856896687540C068D66886EA000802F1100009221B268D4F4FEA89
:20A0C000136C1CF807C0C4F3074E1EF807E04FEA0E4E4EEA0C6CC5F3072E1EF807E04CEAB8
:20A0E0000E2C5FFA88FE1EF807E04EEA0C0C4FEA146E1EF807E0C5F3074919F807904FEA59
:20A10000094949EA0E6EC8F3072919F807904EEA092E5FFA83F919F8079049EA0E0E4FEA37
:20A12000156919F80790C8F3074A1AF807A04FEA0A4A4AEA0969C3F3072A1AF807A049EA2E
:20A140000A295FFA84FA1AF807A04AEA09094FEA186818F80780C3F30743DB5D1B0443EA22
:20A160000863C4F30724E45D43EA0423ECB2E45D44EA03082CF07F33DB0973430CF07F34CE
:20A180008CEA44055D4093EA440383EA356383EA3C4383EA3C2350F8044B63402EF07F34D7
:20A1A000E40974430EF07F358EEA450C84EA0C0C94EA450484EA3C6484EA3E4484EA3E2465
:20A1C00050F8045B6C4029F07F35ED09754309F07F3C89EA4C0E85EA0E0E85EA4C0585EA76
:20A1E0003E6585EA394585EA392550F804CB8CEA050528F07F3C4FEADC1C06FB0CFC08F066
:20A200007F3E88EA4E098CEA09098CEA4E0C8CEA396C8CEA384C8CEA382C50F804EB8EEAC2
:20A220000C08521E7FF44BAF220ED25DC5F30746F65D360446EA0262C8F30726F65D42EA41
:20A240000622DEB2F65D3243466872402E0EF65DC8F3074C1CF807C04FEA0C4C4CEA066673
:20A26000C3F3072C1CF807C046EA0C265FFA84FC1CF807C04CEA0606D0F808C08CEA0606B0
:20A280004FEA186C1CF807C0C3F3074E1EF807E04FEA0E4E4EEA0C6CC4F3072E1EF807E0F0
:20A2A0004CEA0E2C5FFA85FE1EF807E04EEA0C0CD0F80CE08EEA0C0C1B0EDB5DC4F307445E
:20A2C000E45D240444EA0363C5F30724E45D43EA04235FFA88F4E45D234300685840086025
:20A2E0004A608E60C1F80CC0BDE8F08700000000781B00201C18002000B583B07B480178FA
:20A300008DF8001040788DF801000A4878442430017A8DF80210417A8DF80310817A8DF823
:20A320000410C07A8DF80500062100A800F0BCF803B000BD941D000080B56D4890F820100F
:20A34000022909D0032901D0052923D1002180F820104FF44051E5E0C07BF22804D0F42833
:20A3600012D0F62808D001BD62480078002811D1BDE80140FAF750BE5E480078002809D116
:20A38000BDE80140FDF766B85A480078002808BFFFF7FAF801BD10B5022000F03EFC544C65
:20A3A00060840246E021544801F038FD94F8200010B1012803D019E0BDE8104022E0E07BFA
:20A3C000F22804D0F4280CD0F62805D010BD49480078002815D15FE046480078002810D172
:20A3E0005EE04448007800280BD151E0022000F087F8002084F820004FF44051022000F0B3
:20A4000088FB10BD10B53A4C608C38B121463A4A12F8013BCB73491C401EF9D1E07BF1285C
:20A4200018D0F2281ED0F42817D0F52806D0F6281DD0F72806D0F82808D01DE0BDE810404C
:20A44000FDF7EEBEBDE81040FDF7F5B9BDE81040FDF700BABDE810404EE7264800780028EA
:20A4600015D115E023480078002810D114E02148007800280BD113E0022000F041F80020DE
:20A4800084F820004FF44051022000F042FB10BDBDE81040FFF778B8BDE81040FAF7BCBDB6
:20A4A000BDE81040FCF7D6BF10B50C462246A02101F0A0FC2146012000F08CFB30210120E1
:20A4C00000F015FB0A48032180F820100B488168091B81600021017310BD0548002180F8D5
:20A4E00020104FF44051022000F013BBFE3F00080437002088370020C43500204837002041
:20A5000080B518B1022807D00AD301BD10210120BDE8044000F0EBBA1021012000F0E7FAAE
:20A520004FF480510220BDE8044000F0F2BA000080B501F049F94FF480414FF0006001F064
:20A5400057F901F043F94FF4A06001F0F9F8192001F044F91B2001F041F91B208DF80000CC
:20A5600000208DF801008DF8020001208DF8030000A801F0EAF819208DF8000001208DF826
:20A58000020000A801F0E1F801BD6B4A00284FF48071104601D000F000BE00F0FCBD80B5C5
:20A5A0000120ADF80000102004E080B50120ADF8000048208DF8030003208DF8020000A983
:20A5C0005E4800F080FD01BD70B582B004460121012000F0FCFF0121594800F0E5FD102016
:20A5E000ADF800008DF8030003208DF80200534D00A9284600F067FD00221021284600F0C8
:20A60000CEFD0220ADF8000010208DF8030003208DF8020000A9284600F055FD01220221A7
:20A62000284600F0BCFD012C06D101220121284600F0B5FDFFF7B3FFFF26FF20401EFDD192
:20A64000012C04D100220121284600F0A8FD00220221284600F0A3FD761EFDD1012C07D107
:20A6600001220121284600F09AFD9F26761EFDD101220221284600F092FD0220ADF800007F
:20A6800048208DF8030003208DF8020000A9284600F019FD012C08BFFFF787FFFDF7BCFCE7
:20A6A00073BD10B582B00021254800F07DFD0021012000F08CFF1020ADF8000004208DF840
:20A6C000030003208DF802001C4C00A9204600F0FAFC0120ADF8000004208DF8030000A955
:20A6E000204600F0F0FC0220ADF8000004208DF8030000A9204600F0E6FCE020ADF800001F
:20A7000004208DF8030000A90E4800F0DCFC4FF42040ADF8000000A9204600F0D4FC4FF46C
:20A720008040ADF8000004208DF8030000A9204600F0C9FC13BD000000140140000C0140D2
:20A7400000013000000801402DE9F84F4BF68F78684D48F60F7B40F68F77674CDFF89C916A
:20A76000DFF89CA123E0300404D5206838402060FEF7E6FD206808EA00002988CA0448BF5D
:20A7800080F48050890444BF80F4005080B22060206848F6BF7108406988CA0648BF80F0F9
:20A7A0001000890644BF80F0200080B22060606CAAF80000000460D547F6FF706064BAF8EC
:20A7C000000010F00F0089F8000035D1206800F440502880206800F030006880206808EA25
:20A7E000000080F400502060206848F6BF71084080F020002060BAF80000C00620680FD4E4
:20A800000BEA00002060FEF743FD20684FF408410842AFD0206838402060FEF707FDA9E7A8
:20A8200086B2300605D520680BEA00002060FEF72FFD300597D5EDE754F820108EB231044C
:20A840000AD554F82010394044F820102D4901EB800050F8040C80473006A8D599F8000073
:20A8600054F820100BEA010144F82010264901EB800050F8040C804799E7BDE8F18F2DE944
:20A88000F84FDFF8809040F68F75DFF86CB01B4F47F6FF781A4CDFF874A024E0CAF80080A8
:20A8A000208800F00F0038705BF820108EB2310409D55BF8201029404BF8201009EB8000A0
:20A8C00050F8040C804730060DD538785BF8201048F60F7211404BF820100B4901EB8000CB
:20A8E00050F8040C8047DAF8000020800004D5D4BDE8F18F80370020005C004089370020A2
:20A90000863700202036002004360020445C004067490870704766480078704700B585B004
:20A9200001214FF4006000F052FE0121042000F04EFE01F039F85F48842101806020ADF87C
:20A9400000000220ADF808000120ADF8020000A801F037F8012001F06EF8012001F055F8C1
:20A9600005B000BD2DE9F04182B004460D469046514E707884421FD00021042001F049F8C6
:20A980000021012001F045F8002001F03AF8002001F049F8062C46D8DFE804F00461657865
:20A9A000677622004548016821F0F0010091009941F04001016036E0002C4ED0012C4CD0FA
:20A9C000022C4AD0032C48D0042C01D0052C02D17068A84241D0062CDCD17068A8423CD063
:20A9E000374FBD83C5F34F0038854FF6FF7038833889C0B20090009840F4D0400090009897
:20AA00003881A8F10100FF280DD2A7F820800120307001F008F8388820F001003880012141
:20AA2000012000F0F6FF274801210160707828B1042803D0052801D0072809D144B11F48FB
:20AA4000016821F0F0010091009941F0B001016074707560012000F0D4FFBDE8F3815020F8
:20AA600000F0E4FFDFE74020FAE7502000F0DEFF134FBD830220388448F6A0403883002046
:20AA8000307001210420CCE74020EFE70C4F6420B883B88B40083885642038833889C0B213
:20AAA0000090009840F4D040009000983881BAE7161C0020002C0140F81B00200408014069
:20AAC000102C0140808225420722B421062049E74FF6F8710840DFF884110860704710B4F7
:20AAE000DFF87C2152F8203048F68F145CE010B4DFF86C2152F8203048F6BF742340CC06C3
:20AB000048BF83F01003890644BF83F020039BB210E010B4DFF8482152F820304BF68F7461
:20AB20002340CC0448BF83F48053890444BF83F400539BB242F8203010BC7047DFF82011D5
:20AB400051F820204BF68F731A4082F4405208E0DFF80C1151F8202048F68F6300E0000052
:20AB60001A4041F820207047DFF8F41051F82020520408D551F8202048F68F731A4042F45B
:20AB8000804241F820207047DFF8D41051F82020520608D551F8202048F68F731A4042F0F5
:20ABA000400241F8202070472340194342F8201010BC704738E0294A126892B202EBC00081
:20ABC000284A37E03BE02549096889B201EBC00024493AE0214A126892B202EBC000224A42
:20ABE0002AE01E4A126892B202EBC0001F4A02EB40003F2909D34A091F23194204BF521E7B
:20AC000092B2910241F4004105E04A08C90744BF521C92B29102016070471049096889B27B
:20AC200001EBC000114914E00C4A126892B202EBC0000F4A4908490042F810107047074905
:20AC4000096889B201EBC000094951F8100080B2704751F810008005800D7047505C0040FA
:20AC6000005C004008600040046000400C600040006000400106090C41EA10207047000072
:20AC8000008040C020A060E0109050D030B070F0088848C828A868E8189858D838B878F834
:20ACA000048444C424A464E4149454D434B474F40C8C4CCC2CAC6CEC1C9C5CDC3CBC7CFC94
:20ACC000028242C222A262E2129252D232B272F20A8A4ACA2AAA6AEA1A9A5ADA3ABA7AFAB4
:20ACE000068646C626A666E6169656D636B676F60E8E4ECE2EAE6EEE1E9E5EDE3EBE7EFE14
:20AD0000018141C121A161E1119151D131B171F1098949C929A969E9199959D939B979F993
:20AD2000058545C525A565E5159555D535B575F50D8D4DCD2DAD6DED1D9D5DDD3DBD7DFDF3
:20AD4000038343C323A363E3139353D333B373F30B8B4BCB2BAB6BEB1B9B5BDB3BBB7BFB13
:20AD6000078747C727A767E7179757D737B777F70F8F4FCF2FAF6FEF1F9F5FDF3FBF7FFF73
:20AD800007000000000000000100000000000000020400000A000000060000000000000095
:20ADA0000700000000000000020FB70007000108000000000500000000000000020FB700E7
:20ADC00007000108000000000500000000000000020FB70007000108000000000500000081
:20ADE000000000000600000000000000078000000000000080B5B0F1804F06D048498842F0
:20AE00000AD0484988420ED001BD0121012000F0F9FB002101200CE00121022000F0F2FBEB
:20AE20000021022005E00121042000F0EBFB00210420BDE8044000F0E5BB0A8882854A88A5
:20AE40000285028802F08F02028002888B88C988194385E070B4038C4C880CB1012C29D1C2
:20AE60002E4D7D44B635028B35F81460324005EB44052D892B40002C048C0BD143F232357D
:20AE80002C4004840C8822438C888486C98841F001010CE043F223352C4004840C8842EAF6
:20AEA00004228C880487C988090141F010010B4302832FE0022C01D0032C2BD1174D7D44FF
:20AEC0005A35828B35F81460324005EB44052D892B40022C048C0DD143F233252C4004844C
:20AEE0000C8822438C888487C9884FF4807444EA01210DE042F233352C4004840C8842EA25
:20AF000004228C88A0F84040C988090341F480510B438283038470BC704700BFD41100001B
:20AF200000040040000800400185012A818A0CBF41F0010101F0010181827047028B4FF64C
:20AF4000F7731A401143018370470288002912BF42F0020140F2FD311140018070471A40A2
:20AF6000114301807047000080B53E49401A17D04FF48061401A1CD0401A23D0401A2AD03D
:20AF80004FF46841401A30D101214FF4804000F030FB00214FF48040BDE8044000F029BB49
:20AFA00001214FF4003000F02DFB00214FF4003019E001214FF4802000F024FB00214FF4DF
:20AFC000802010E001214FF4002000F01BFB00214FF4002007E001214FF4801000F012FBF9
:20AFE00000214FF4801000F00DFB01BD30B585B004460D46208A4CF6FF710840E988084390
:20B000002082A0894EF6F3110840A98808432989084369890843A081A08A4FF6FF41084007
:20B02000A9890843A08200A800F088FA0E4884420CBF039802981921484329688900B0FBB1
:20B04000F1F06421B0FBF1F21201130901FB130000013230B0FBF1F000F00F0010432081DC
:20B0600005B030BD0044004000380140028A4FF2FF031A400B881A434B881A438B881A4378
:20B08000C98812E00029818914BF41F4005121F4005181817047002A828A14BF114322EA59
:20B0A0000101818270470282028A11430182704780B50121012000F09CFA00210120BDE851
:20B0C000044000F096BA2DE9F041CB7803F00F02DB0644BF8B781A430B88DCB22CB3D0F852
:20B0E00000C0002401250F2605FA04F707EA0308B84515D14FEA840E06FA0EF82CEA080C3D
:20B1000002FA0EFE4EEA0C0C91F803E0BEF1280F08BF476191F803E0BEF1480F08BF076175
:20B12000641C082CE0D3C0F800C04FF48074A34227D3D0F804C0002401250F2604F108070B
:20B1400005FA07F707EA0308B84515D14FEA840E06FA0EF82CEA080C02FA0EFE4EEA0C0CC0
:20B1600091F803E0BEF1280F08BF476191F803E0BEF1480F08BF0761641C082CDED3C0F850
:20B1800004C0BDE8F0818068FFE70140481E8041C043C00F70470161704741617047002A7A
:20B1A00014BF01614161704770B40D4A1368C0F3034485B2860248BF23F0E06306D4C60253
:20B1C00043BF032606FA04F4A343AB4321B180024CBF43EA05432B43136070BC70470000E0
:20B1E000040001404268454B1A400B681A430B7942EA032242608268414B1A40CB681A43CF
:20B200008B681A434B7942EA43028260C26A22F47002097C491EC9B242EA0151C162704754
:20B220000029816814BF41F0010121F0010181607047816841F008018160704780680006A2
:20B24000C00E07E0816841F004018160704780680006800E00F0010070470029816814BF79
:20B2600041F4A00121F4A0018160704770B4032407250A290AD3A1F10A067443C668A540B7
:20B2800026EA0505A3402B43C36007E04C430669A54026EA0505A3402B43036105231F241C
:20B2A000072A08D2521E5A43436B9440A34391401943416312E00D2A08D2D21F5A43036B3E
:20B2C0009440A34391401943016307E00D3A5A43C36A9440A34391401943C16270BC70473E
:20B2E000C06C80B2704707490028086814BF40F4000020F40000086070470000FFFEF0FF2B
:20B30000FDF7F1FF0824014000680140481E8041C043C00F704700007047FEE7FEE7FEE71D
:20B32000FEE7704770477047FBF7B2BB704770477047704770477047FBF7F0BA7047704750
:20B3400070477047FBF76EBB202000F0EAB84FF4007000F0E6B829484FF400510160704734
:20B3600027480078032801D1FBF747BBFEF7B5BD4FF4001000F0D5B8FBF72ABB7047FFF73A
:20B380007EBA00F03FBC704770477047704780B51C48018821F0010101801B4800780128F4
:20B3A0000CD1FFF7B8FA012802BF00220021022002D0002200210320FFF7D4FA01BD704748
:20B3C00080B51048018821F0040101801B2000F005FA0D48007880B90C480168491C01600D
:20B3E0000B48026822F0F0020092C90700994CBF41F0400141F0B001016001BD04000240CD
:20B40000E0360020102C0140F81B0020703700200408014070477047FBF720BB7047704789
:20B42000704770477047704770477047704770477047704710B50446002100F054F800205A
:20B4400020606060A060E0603848241A0CD0143C0FD0143C12D0143C15D0143C18D0143CB4
:20B460001BD0143C1ED010BD3148016841F00F011CE02F48016841F0F00117E02C480168E1
:20B4800041F4706112E02A48016841F470410DE02748016841F4702108E02548016841F475
:20B4A000700103E02248016841F07061016010BD0268204B1A408B681A430B6A1A430B6970
:20B4C0001A434B691A438B691A43CB691A434B6A1A438B6A1A430260CA6842600A6882602E
:20B4E0004968C16070470029016814BF41F0010121F0010101607047002A026814BF114345
:20B5000022EA010101607047406880B2704700E007E0094909680840401E8041C043C00FB1
:20B5200070470349086070470000000008000240040002400F80FFFF0000024010B4374946
:20B540000A6812F00C0203D0042A01D0082A24D0334A02600B68184A7A445C320468C3F34F
:20B5600003139B5C24FA03F343600C68C4F30224A45CE34083600B684468C3F3C2239B5CFF
:20B5800024FA03F3C3600968C1F381318918097CB3FBF1F1016110BC70470A68C2F3834216
:20B5A000921C0B68DB0302D41E4B5A43D1E70B689B03F9D41A4BF8E7FC0A00001A4A002943
:20B5C000116814BF084321EA000010607047174A0029116814BF084321EA0000106070474F
:20B5E000134A0029116814BF084321EA000010607047104A0029116814BF084321EA0000D7
:20B60000106070470C4A0029116814BF084321EA00001060704709490870704704100240E4
:20B6200000127A0000093D0014100240181002401C1002400C1002401010024007100240E1
:20B640000001010001000001010000010001010001000001000101000001010001000001DA
:20B660000100000100010100000101000100000100010100010000010100000100010100BA
:20B6800001000001000101000001010001000001000101000100000101000001000101009A
:20B6A00000010100010000010100000100010100010000010001010000010100010000017A
:20B6C00001000001000101000001010001000001000101000100000101000001000101005A
:20B6E00000010100010000010100000100010100010000010001010000010100010000013A
:20B70000000101000100000101000001000101000100000100010100000101000100000119
:20B720000100000100010100000101000100000100010100010000010100000100010100F9
:20B74000314908433149086070472DE9F04105780121C2787AB32D4A126802F4E062C2F55E
:20B76000E062120AAB10DFF89C8058F8237005F00305ED00FF26AE40B7434478C2F1040E62
:20B7800004FA0EFC90F802E00F2424FA02F202EA0E0242EA0C021201AA4032403A4348F890
:20B7A0002320007842111A4B00F01F0001FA00F043F8220006E06811104A05F01F03994016
:20B7C00042F82010BDE8F08100F067BA00F063BA000100F06EBA0F49086070474111084A97
:20B7E000012300F01F0003FA00F042F821007047094A1140084309490860704780E100E076
:20B8000080E200E000E400E00000FA050CED00E000E100E000EF00E080FFFF1F08ED00E048
:20B82000576861742061726520796F7520646F690000000000000000000000000000000043
:20B840000000000000000000000000000000000000000000000000000000000000000000E8
:20B860000000000000000000000000000000000000000000000000000000000000000000C8
:20B880000000000000000000000000000000000000000000000000000000000000000000A8
:20B8A000000000000000000000000000000000000000000000000000000000000000000088
:20B8C000000000000000000000000000000000000000000000000000000000000000000068
:20B8E000000000000202020202020202020202020200020202020202020202020202020014
:20B900000202020202020202020202020200020202020202020202020202020001010001F0
:20B920000101000000000101010001010001010100000000010101000101010101010100F3
:20B940000000010101000202020202020202020202020200020202020202020202020202B2
:20B960000200020202020202020202020202020001010001010100000000010101000101A1
:20B9800000010101000000000101010002020202020202020202020202000202020202027B
:20B9A000020202020202020080B501214FF40060FFF71FFE00214FF40060BDE80440FFF7C9
:20B9C00018BE10B4DFF884100A88DFF8843000241C60D2B2048842EA04220A8042881A6075
:20B9E00082889A6002895A604289DA60DFF86420FFE783891360C3895360C088088410BC9A
:20BA00007047DFF8541008607047DFF8501008607047DFF84C20012911880CBF084321EA98
:20BA20000000108070470F490860704707490A8840F67F7305E00C49086070470A884FF212
:20BA4000FF331A4042EA002008807047182C014010842542A880254200802542BC8825422E
:20BA60000C2C01400C8025422C8325422DE9F04100F10801026801EB8202406800F001038D
:20BA80004008400002EB80004FF0000CE646002401250CE01CF8018BBE4206D006F8018B04
:20BAA000641C24B2002CF7D40125BE4212D1824201D1BDE8F08152F8046B03B14E4452F83B
:20BAC000047BBF19F1E7D1F800C08C44091D51F804EBE644F445F6D065B11CF9014B0025BB
:20BAE00006E0D1F800C08C44091D51F804EBE644F445F6D0002CCDD4002CD5D4BE4218BF07
:20BB0000F4451FBF1CF8018B06F8018B641E24B2F2D1CAE780B50F49401A0FD04FF4784156
:20BB2000401A15D101214FF48050FFF762FD00214FF48050BDE80440FFF75BBD01214FF4AB
:20BB40008040FFF75FFD00214FF48040FFF75AFD01BD000000380040028802F441520B8886
:20BB60001A434B881A438B881A43CB881A430B891A434B891A438B891A43CB891A43028052
:20BB8000098A018270470029018814BF41F0400121F0400101807047002A828814BF1143FC
:20BBA00022EA0101818070470029818814BF41F0040121F004018180704700001E480D49FA
:20BBC0007944303101600C4979442C3141600B4A7A4428328260C160016141618161C1615E
:20BBE000074A7A441A32026241628162C1620163416370472905000011D8FFFF29050000DB
:20BC00002105000038B50D4C0D48016821800D4D21882A881140490505D54FF6FF31016055
:20BC2000094840688047208829880840000448BFFEF78AFD31BD00000436002086370020F7
:20BC4000445C004084370020481B002030BF704720BF704740BF7047BFF36F8F7047BFF39B
:20BC60004F8F7047BFF35F8F704701DF7047EFF31480704780F31488BFF36F8F7047EFF3BC
:20BC80000980704780F309887047EFF30880704780F30888704762B6704772B67047EFF33E
:20BCA0001080704761B6704771B67047EFF31380704780F311887047EFF31280704740BA7D
:20BCC000704700BA704700004AB38B0707D011F8013B00F8013B521E21D08B07F7D1830718
:20BCE0001ED1103A07D330B4B1E83810103AA0E83810F9D230BC530724BFB1E80810A0E825
:20BD0000081044BF51F8043B40F8043BD20724BF31F8022B20F8022B44BF0B780370704702
:20BD2000083A07D3B1E80810083A40F8043B40F804CBF7D25307E4E762F30F2262F31F424C
:20BD4000401810F0030308D0C91A1FD3DB0748BF00F8012D28BF20F8022D130030B414464A
:20BD60001546103928BF20E93C00FAD8490728BF20E90C0048BF40F8042D890028BF20F8DD
:20BD8000022D48BF00F8012D30BC7047C91818BF00F8012DCB0728BF00F8012D7047000030
:20BDA000201000E0301000E0401000E0501000E0241000E0341000E0441000E0541000E033
:20BDC000281000E0381000E0481000E0581000E0000000000004000000080000000C00008B
:20BDE000040000000500000006000000070000000000000010B4104B03EB4101521C52100E
:20BE00000AD010F8013B10F8014B43EA042321F8023B891C521EF4D110BC7047064B03EB6A
:20BE20004101521C521005D051F8043B20F8023B521EF9D1704700000060004080B5FEF783
:20BE400077FBFBF74DFDFBF7BFFD401E8041C00F07490870074800780328FBD10820FFF7F4
:20BE6000B7FC0548006880470020FFF7B1FCF1E788370020E0360020881900200E49086063
:20BE800070470C49002801D188607047012808680CBF40F0010020F00100086070470549EA
:20BEA0000028086814BF40F0020020F0020008607047000010E000E014E000E00C48016853
:20BEC00021F0010101600B494A6901EB42039B88436001EBC22101F21C01C160016841F056
:20BEE000010101600448018841F400510180704758000240000800200C38014080B500F0E0
:20BF000027F902000023DB431068984204D011000220ABBE002010605068984204D0111DD8
:20BF20000220ABBE0020506001BD000080B50120FEF72BFB06480121016000210160416083
:20BF40004FF4E051034A11800160002002BD0000405C00408437002010B5084979441C3178
:20BF6000074C7C441A34A14206D0081D0A68511888470146A142F8D110BD00BF7C000000DD
:20BF8000A80000000902270001010080320904000003FFFFFF040705810240000007050225
:20BFA0000240000007058302400000002603530054004D006900630072006F0065006C00D3
:20BFC00065006300740072006F006E0069006300730000000BE050F8041BCB0744BFA9F1D6
:20BFE00001035918002341F8043B121FFAD150F8042B002AEFD17047DDFFFFFF741B0000B4
:020000040800F2
:20C00000181C00200000000065FAFFFF020000000200000058010000B10200000008002037
:20C020001714000025000000082000E00C2000E0102000E0142000E0182000E01C2000E044
:20C04000202000E0242000E010B50446044979440E31044878440C3000F014F8204610BDD1
:20C06000BC000000AC0000001A03530054004D00330032002000530054004C0069006E00F8
:20C080006B00000038B504460D46AC4205D0206820188047241DAC42F9D131BD00F064F82E
:20C0A000002801D0FFF758FF0020FFF7C7FE00F056F800000000000001020304010203040D
:20C0C0000607080902040608120100020000004083044837000101020301000080B5FFF7A0
:20C0E0000DFF024A11001820ABBEFBE72600020000FFFF0000FFFF003133133333313313DC
:20C1000010035300540020004C0069006E006B008599FFFFA9FAFFFFC1D7FFFFFEF70CB9AA
:20C12000FEF739B9FDF745BFC046C046C046C046FFF7B4FF07463846FFF7D0FFFBE70000ED
:20C1400000480000C400000000080000C400000000487047001C00200022FFF7F1BD80B5D1
:20C16000FFF7E8BF0403090401207047FB0002080008F00001127A81008100810081008127
:20C1800000810081008100810081008100810081008100810081008100810081008100818F
:20C1A0000081008100810081008100810081008100810081008100DE007E637C777BF26B6A
:20C1C0006FC53001672BFED7AB76CA82C97DFA5947F0ADD4A2AF9CA472C0B7FD9326363F30
:20C1E000F7CC34A5E5F171D8311504C723C31896059A071280E2EB27B27509832C1A1B6E31
:20C200005AA0523BD6B329E32F8453D100ED20FCB15B6ACBBE394A4C58CFD0EFAAFB434D39
:20C22000338545F9027F503C9FA851A3408F929D38F5BCB6DA2110FFF37ED2CD0C13EC5F9F
:20C24000974417C4A77E3D645D197360814FDC222A908846EEB814DE5E0BDBE0323A0A4948
:20C2600006245CC2D3AC629195E479E7C8376D8DD54EA96C56F4EA657AAE08BA78252E1C90
:20C28000A6B4C6E8DD741F4BBD8B8A703EB5664803F60E613557B986C11D9EE1F89811695E
:20C2A000D98E949B1E87E9CE5528DF8CA1890DBFE6426841992D0FB05401BB16FA00000335
:20C2C000D10009C6006300AB001B008004C8006968360020903600203200A00F7017401F75
:20C2E0001027E02EB036803E5046204E0852F055D859C05DA86190657869606D0100AB000C
:20C30000C60071018C01370252026D02180333030100AB00C60071018C01A7015202FD029F
:20C32000180333030100AB00C60071018C0137025202FD021803C30331109A000003FD00F3
:20C3400013741A0020781A0020141C0020C00CC0180F800F70D4000008FD0002018004FC0C
:20C360000001C020FC0000C0D6000004F9000026F900001AFD0004C41B00201AF9000010F1
:20C38000F9000012F9000027FD000002F9000003F1000002F1000006CD000040FA00000185
:20C3A000FD000002FD000004FD000008FD000010FD000020FD000040FD000080FD00001B7C
:20C3C000FD001536A58D95BD87AFB79FA38B93BB81A9B199F00000FFFFF100181A033000D1
:20C3E000300030003000300030003000300030003000300031FD000001F9000302000080B0
:20C40000F80005083001400007FA00F8FF0E1E009E040401000005F80DF807F801CDCDCD72
:20C42000FFFFFFFFFFFFFFFFFFFFFFFFFFFFFFFFFFFFFFFFFFFFFFFFFFFFFFFFFFFFFFFF1C
:20C44000FFFFFFFFFFFFFFFFFFFFFFFFFFFFFFFFFFFFFFFFFFFFFFFFFFFFFFFFFFFFFFFFFC
:20C46000FFFFFFFFFFFFFFFFFFFFFFFFFFFFFFFFFFFFFFFFFFFFFFFFFFFFFFFFFFFFFFFFDC
:20C48000FFFFFFFFFFFFFFFFFFFFFFFFFFFFFFFFFFFFFFFFFFFFFFFFFFFFFFFFFFFFFFFFBC
:020000040800F2
